:100000000C9445230C946D230C946D230C94D62DE5
:100010000C946D230C94312D0C946D230C946D2352
:100020000C946D230C946D230C946D230C94622E10
:100030000C946D230C946D230C946D230C946D2300
:100040000C94692C0C946D230C94372C0C94112C6B
:100050000C946D230C94F22D0C946D230C946D2351
:100060000C94B32C0C946D236841774186419541E3
:10007000A541B441C341D241E141F14100420F42A7
:100080001E422E423D424C425C426B427A428A42C0
:100090009942A842B842C742D742E642F6420543D7
:1000A00015432443344343435343624372438143E0
:1000B0009143A143B043C043D043DF43EF43FF43E9
:1000C0000E441E442E443E444D445D446D447D44E4
:1000D0008D449C44AC44BC44CC44DC44EC44FC44DF
:1000E0000C451C452C453C454C455C456C457C45C8
:1000F0008C459C45AC45BC45CC45DC45ED45FD45B6
:100100000D461D462D463D464E465E466E467F4692
:100110008F469F46AF46C046D046E146F14601476E
:10012000124722473347434754476447744785473C
:100130009647A647B747C747D847E847F9470A4809
:100140001A482B483C484C485D486E487F488F48C9
:10015000A048B148C248D248E348F4480549164986
:100160002749384949495A496B497C498D499E4933
:10017000AF49C049D149E249F349044A154A264AE0
:10018000374A484A5A4A6B4A7C4A8D4A9E4AB04A84
:10019000C14AD24AE34AF54A064B174B294B3A4B20
:1001A0004C4B5D4B6E4B804B914BA34BB44BC64BB2
:1001B000D74BE94BFA4B0C4C1D4C2F4C414C524C3D
:1001C000644C764C874C994CAB4CBC4CCE4CE04CC0
:1001D000F24C034D154D274D394D4B4D5D4D6E4D38
:1001E000804D924DA44DB64DC84DDA4DEC4DFE4DAF
:1001F000104E224E344E464E584E6B4E7D4E8F4E14
:10020000A14EB34EC54ED84EEA4EFC4E0E4F214F76
:10021000334F454F574F6A4F7C4F8F4FA14FB34FCE
:10022000C64FD84FEB4FFD4F10502250355047501E
:100230005A506C507F509150A450B750C950DC5068
:10024000EF500151145127513A514C515F517251A5
:1002500085519851AB51BD51D051E351F6510952DE
:100260001C522F524252555268527B528E52A1520A
:10027000B452C852DB52EE520153145327533B532E
:100280004E536153745388539B53AE53C253D5534B
:10029000E853FC530F54235436544A545D5471545C
:1002A00084549854AB54BF54D254E654FA540D5568
:1002B0002155355548555C55705583559755AB5567
:1002C000BF55D355E655FA550E56225636564A5660
:1002D0005E56725686569A56AE56C256D656EA564E
:1002E000FE56125726573A574F57635777578B5733
:1002F0009F57B457C857DC57F157055819582E580F
:10030000425856586B587F589458A858BD58D158E1
:10031000E658FA580F59235938594D5961597659A9
:100320008B599F59B459C959DE59F259075A1C5A69
:10033000315A465A5A5A6F5A845A995AAE5AC35A1F
:10034000D85AED5A025B175B2C5B415B565B6B5BCB
:10035000815B965BAB5BC05BD55BEB5B005C155C6C
:100360002A5C405C555C6A5C805C955CAA5CC05C05
:10037000D55CEB5C005D165D2B5D415D565D6C5D93
:10038000815D975DAD5DC25DD85DEE5D035E195E1A
:100390002F5E455E5B5E705E865E9C5EB25EC85E92
:1003A000DE5EF45E0A5F205F365F4C5F625F785FFF
:1003B0008E5FA45FBA5FD05FE65FFC5F126029606A
:1003C0003F6055606B6082609860AE60C560DB60C6
:1003D000F16008611E6135614B61626178618F6116
:1003E000A561BC61D261E961006216622D6244625E
:1003F0005A62716288629F62B662CC62E362FA629C
:10040000116328633F6356636D6384639B63B263C8
:10041000C963E063F7630E6425643C6453646B64F2
:1004200082649964B064C864DF64F6640D65256510
:100430003C6554656B6582659A65B165C965E06523
:10044000F865106627663F6656666E6686669D6628
:10045000B566CD66E566FC6614672C6744675C6725
:1004600074678C67A467BC67D467EC6704681C6812
:1004700034684C6864687C689468AC68C468DD68FB
:10048000F5680D6925693E6956696E6987699F69D6
:10049000B869D069E969016A1A6A326A4B6A636AA3
:1004A0007C6A946AAD6AC66ADE6AF76A106B296B69
:1004B000416B5A6B736B8C6BA56BBD6BD66BEF6B23
:1004C000086C216C3A6C536C6C6C856C9E6CB86CCF
:1004D000D16CEA6C036D1C6D356D4F6D686D816D6F
:1004E0009B6DB46DCD6DE76D006E196E336E4C6E05
:1004F000666E7F6E996EB26ECC6EE66EFF6E196F91
:10050000336F4C6F666F806F9A6FB36FCD6FE76F0D
:1005100001701B7035704F70697083709D70B7707B
:10052000D170EB7005711F71397153716E718871E3
:10053000A271BC71D771F1710B72267240725A723E
:1005400075728F72AA72C472DF72F97214732E738D
:10055000497364737E739973B473CF73E9730474CE
:100560001F743A74557470748A74A574C074DB7403
:10057000F67411752C75487563757E759975B4752B
:10058000CF75EB75067621763C76587673768E7647
:10059000AA76C576E176FC76187733774F776A7757
:1005A0008677A277BD77D977F57710782C78487859
:1005B000647880789B78B778D378EF780B7927794F
:1005C00043795F797B799779B379CF79EC79087A38
:1005D000247A407A5D7A797A957AB17ACE7AEA7A13
:1005E000077B237B407B5C7B797B957BB27BCE7BDF
:1005F000EB7B077C247C417C5E7C7A7C977CB47CA2
:10060000D17CEE7C0A7D277D447D617D7E7D9B7D56
:10061000B87DD57DF27D107E2D7E4A7E677E847EFC
:10062000A17EBF7EDC7EF97E177F347F527F6F7F95
:100630008C7FAA7FC77FE57F028020803E805B8021
:1006400079809780B480D280F0800E812C8149819E
:1006500067818581A381C181DF81FD811B82398210
:10066000578276829482B282010002000400080060
:10067000100020004000800000010002000400FF84
:1006800000FF00FF00FF00FFFF00FF01FCFEFFF87E
:10069000F7FCFAF2F2F0F1EBE8E9EFECE5E8E7E974
:1006A000E6E8E6E6E7E9E5E4EDE5EFE1EDE1EF04B4
:1006B000B704FAD7E7D32913FD0E0D2D15234213E6
:1006C0002736462E264F274B3B384A3B5046544947
:1006D00050594A534F4B4945423F3C393835312EEA
:1006E0002B282522211E1D1E1C1C1B1B1918170F31
:1006F000120D0D0B0104F9F5E1D9E6D0CFCEC1C240
:10070000BDB1B0ABACAE9CA4AA9593999894888BDC
:100710008F85848C85878D8F979A9EA3A7ABADB16B
:10072000B5B8BBBFC0C3C5C8C9CBCFD1D4D6D9DD3E
:10073000DEE0E3E5E7E9EAECEFF1F1F3F4F6F7F9EF
:10074000FBFCFEFF01030507080D0E0D1517181C15
:100750002325242A2F2E2F3838383A403E3B454453
:1007600044464C4C454B52494A51494C5049484DDE
:100770004F4B4B494D4D4D4E484D4D514B475049B8
:100780004F4A4949434D48424444444242433C3F16
:10079000403B3E3E3E37383F3935373530322E2CE0
:1007A000292624211F1C1A181614110F0E0B0906D6
:1007B0000402FFFEFCFAF9F7F6F5F4F3F2F0EFEEBF
:1007C000EDECEBEAE9E8E7E6E5E4E3E2E2E0E0DAD3
:1007D000D8D9D3D1CECCCAC8C3C1BEBCBAB5B5B0C6
:1007E000B0AEABA9A7A8A5A4A3A09FA09C9E9E99CC
:1007F00098989C97989C99989A98989C999A9C9B61
:10080000989B9F9D9C9E9FA0A1A3A8A8ACAFB3B7A7
:10081000BBBFC1C5C8CACED1D4D7DADCDFE1E5E7BA
:10082000EAECEFF1F3F5F7F9FBFEFF000204050631
:1008300008090B0C0D0E1012131516181B1E20257F
:1008400029292D313335373C3F3F43444648494BF6
:100850004C4E4E5152535555565656595A585A5A4F
:100860005E5E585C5D5C5B5C5B59595656555453F3
:10087000535251504F4F4B4A4A4846444342403EE0
:100880003E3C3A38363432302E2D29262524201F7E
:100890001E1B1A181613120F0E0C0907060300FE72
:1008A000FEFCF8F6F5F3F0EEEDECEBE8E6E6E5E459
:1008B000E1E0E0DEDDDBDBD9D8D8D5D5D3D2D3D2A9
:1008C000D1D1D1D1D0CFD0D0CFCFCFCFD0CECDCE30
:1008D000CECFCFCED0D0D0D1D1D3D3D4D4D6D7D7FA
:1008E000D9D9DADADBDCDCDDDEDFE1E1E1E3E4E526
:1008F000E5E6E8E9EAEAEDEEEEEFF0F1F3F3F5F61E
:10090000F5F6F7F9F9F9FAFBFCFDFF000002020326
:1009100005060607080909090B0B0C0C0C0C0D0D3C
:100920000D0D0E0E0E0F0E0F0E0E0F0F0F0E0E0EE4
:100930000E0F0E0E0E0D0D0E0E0C0C0D0C0C0C0BE6
:100940000B0B0B0A0A090909090808080808080816
:100950000808070707070506050505040403030340
:100960000303020302020201020202020101010169
:100970000000000000FFFFFFFFFFFFFFFFFEFFFF83
:10098000FEFEFEFEFEFEFFFEFEFEFEFEFDFDFEFE88
:10099000FDFEFEFEFEFEFEFEFEFEFEFEFEFEFEFE78
:1009A000FEFEFEFEFEFEFEFEFEFEFEFEFEFEFEFE67
:1009B000FEFEFEFEFEFEFEFEFEFEFEFDFEFDFDFE5A
:1009C000FEFEFEFEFEFEFEFEFEFEFEFFFFFFFFFF42
:1009D000FFFFFFFFFFFFFFFFFFFFFFFFFFFFFFFF27
:1009E000FFFFFFFFFFFFFFFFFFFFFFFFFFFFFFFF17
:1009F000FFFFFFFFFFFFFFFFFFFFFFFFFFFFFFFF07
:100A0000FFFFFFFFFFFFFFFFFFFFFFFFFFFFFFFFF6
:100A1000FFFFFFFFFFFFFFFFFFFFFFFFFFFFFFFFE6
:100A2000FFFFFFFFFFFFFFFFFFFFFFFFFFFFFFFFD6
:100A3000FFFFFFFFFFFFFFFFFFFFFFFFFFFFFFFFC6
:100A4000FFFFFFFFFFFFFFFFFFFFFFFFFFFFFFFFB6
:100A5000FFFFFFFFFFFFFFFFFFFFFFFFFFFFFFFFA6
:100A6000FFFFFFFFFFFFFFFFFFFFFFFFFFFFFFFF96
:100A7000FFFFFFFFFFFFFFFFFFFFFFFFFFFFFFFF86
:100A8000FFFFFFFFFFFFFFFFFFFFFFFFFF0000145F
:100A90000B0808F503F2A8BBB8B8C8B0B3BEB5C917
:100AA000CDADE3E5DFF11B2734583A402C5E6452AC
:100AB00058374048535654455C2F15584423231B40
:100AC000200B011F160F0B01FBE5DED1F2F0C6EB88
:100AD000D7AFC5DBD2A9A6A5999F9FA4A6BBC0B0DE
:100AE000B4B4B8BAC5CACEC6D8F5FC281F20403F5A
:100AF0003A54645D6863655F5A5753544E4E473BA2
:100B00002F281D0C0BFEFEFAF0F7F1E1DFE3CDDF3D
:100B1000E3C3CFC6B4B4AAA4A0A8ACB6B5C4D0C829
:100B2000F1F8FB1A2F27132B2F212D1B011E161650
:100B3000231D190C180708180705FEF612F5FD0A03
:100B4000F717060113100618231E1C15291E17205F
:100B5000140E130C0402EFF8EEE7E6E3E2D7E3D657
:100B6000D1D6D5D2CFDEDBE5E4E1F7E6EDF5F3FD56
:100B7000E6FAFEE80504FB0903070811140D140A40
:100B800011261D1A1F24311A242D2433271B1E3031
:100B90002E221421230D0D010400FCECE5F3E3E803
:100BA000E0D3D5BFCAD8C0C4BEBFCFD2CBC4DEDE6F
:100BB000E0E4E6F9EDF315FEFA03080D020E081B5A
:100BC00016072723142213172C12272F1E1D263633
:100BD000222525301F15251F2E111B1F0E1B07EF69
:100BE000FEF6E5E8D2E2CEC7DDC9CFCDD9D1C5CE7C
:100BF000D9DADADFD7DCEEE9E3F8F2EDF8EFFC0260
:100C0000F90A0A010C01132111281D1B3529242C76
:100C100027323420303D2E222B231E20111A130A96
:100C200008F9FF00FBF2E9E7D6E7E8D7D6D4D2D03F
:100C3000D2CAC8D7E1D4DBE1D9F2E9DD04EEE5069A
:100C4000FFFA0FFC021C06162821111A18191D0A9A
:100C5000121A1F140E141E0E08100F150C0B12057D
:100C600015200F160B0B0AF90B0AF703F0EBF3EA4A
:100C7000ECEBF0DFE8EADBECDCE2F2EAF2EBF2EAE2
:100C8000F5FEE6FFFCF3F8F909FA0B03F912FB078E
:100C90000BF4121206050622040A1A131708190E7D
:100CA00016120E1A0E211C120F1912051200060D33
:100CB00008FCF702FE06EBEFFBEAE9E7EFE3E6EB01
:100CC000E5EBEBDFEEF5D4F0F8D9EBEBECF0F3FF6E
:100CD000F0FC06F9FC0E0705080A0F0506091803C3
:100CE0000711090D0516100D101411140D0F1B0C12
:100CF00018131B091317F916070107FBFA00F3F085
:100D0000FEF2F6F0ECF3ECEBF4E6F0FCE5F3F5E3E1
:100D1000F4F7EAF0FCF0E9FCEDEF00F4F3FB03FA82
:100D2000FBFAFE07FE000805FE070D140C12201644
:100D3000191E1F17191D2317091B140D120C050A64
:100D40000B03FB01FBF1FFF4F8ECECEDDDEAE6E868
:100D5000E9DBDBE5E2E3ECEADFE9FAE6F2FBF6FBEE
:100D6000F9030803020C07090B0D1305020F170402
:100D70000E0EFF140A0A07090C050E06090D0F0ACC
:100D80001111060C0B0D0C060805FF0A01F9FBF802
:100D9000FAF6F8EEEDF2F3EEEBF5EBE5F4F1E8F64A
:100DA000F1EBF1F5F5F0F6F6F4F5FBFAF900FB01DD
:100DB0000C06FD09140806120E080A1112090E137A
:100DC000100F110E100F140F080F080906060A065F
:100DD00004F8FF00F8F6F6F9EBEFFBEFF1EFECEFBC
:100DE000E4EFF2EAF3E7EDEFECF8F7F5F6FAFB01E2
:100DF000FFFDFE0209FE020D05000A07080B0307AE
:100E00000A04060D04060C050607080E050A0E095D
:100E10000D050D0C070D0608060104FF02FEFEFF7E
:100E2000F6F9F1F4F8EEF5F1EEEEF0F1ECF9F3F19C
:100E3000F1F3FEF6F4F8FBF9FBFEFA01FEFC09FF04
:100E40000107030401080502100BFD0D0A06120834
:100E50000E120E0F050C100B09070A0506070305F5
:100E600000F800FEFBF9F2FAF2F3F7F3F5F0EEF218
:100E7000F4F4F3ECF2F8F3F3F4F8F5F7F9FB01F915
:100E8000FD05FF0803000E03030705080507050617
:100E900008FE0901000FFF0207050806030C0805FC
:100EA0000F050D09011004010B0400010000FEFDF7
:100EB000F9F3F9F4F3F5EFF0F0F8F1EDF3F4F6F8F7
:100EC000F5F4FBF6F7FCFEFCFC02FF03040205024E
:100ED00004060808040A08080F070A0A0A0C0A0E82
:100EE00008090A0D0A030805010202FDFEFBF8FFCE
:100EF000F7F7FBF8F7F6FAF3F4F5F7F6F3F6F4F68E
:100F0000F1F8F6F6F7F9FEF6FFFDF80201FF02012F
:100F10000207070606080A060A0B080809080A0A53
:100F2000010904010706020205FF06050103010489
:100F30000401FFFFFEFBFD01FBF5FDFAF4F8F8F7F5
:100F4000F1F5F6F2F6F4F5F4F8F9FAFEF8FEFDFD27
:100F500002010500070703080906060A090A06092F
:100F600008050B070807060606070107010003032B
:100F7000FFF901FEFDF9F9FEFBF6F9FBF8F8F4F7CD
:100F8000F9F8F8F6F5F9F8F8FAFDFDFBFCFE02FCBD
:100F9000FA0203FE00050203060806060902070A14
:100FA000070806080307070502FF07010200FD0303
:100FB000FCFF01FDFFFEFDFEFFFEFDFBFDFAFE0056
:100FC000FBFEFAF9FBFDFAF700F9F8FDF6FBFDFA76
:100FD000F9FDFFFAFDFFFF050100060504050806FF
:100FE000070A06070704070907060306050003FDAD
:100FF0000001FBFEFCFBFBFBFAF9F9F8F9FBFAF840
:10100000FBFBFAFCFDFCFDFCFDFEFD0000FD02000B
:10101000FF03FD02050005050200040603030105A8
:10102000010104010302FE0102FE03FDFF01FD00B8
:10103000FEFEFCFF01FFFC0000FDFDFDFFFDFFFFCC
:10104000FCFEFEFEFFFEFD01FEFB00FFFFFEFD00BD
:1010500000FEFF0000000101010301020202000284
:1010600002010204FF0005FF03010001FD0101FE72
:10107000FEFF00FEFDFEFDFDFEFCFBFDFDFDFCFD9B
:10108000FEFDFFFDFD00FFFD0000FEFFFE02010171
:101090000200040301010301020401030000010036
:1010A000010000FF0200FF01FFFE0000FF00FEFC48
:1010B000FEFFFEFCFEFFFBFDFFFDFFFEFDFFFFFD53
:1010C000FE00FFFF000100FFFF02FF02020003011C
:1010D0000202010201000200FF0100FF00FE00FF0A
:1010E000FE00FEFFFEFFFEFC01FCFDFFFBFFFDFE20
:1010F000FFFCFEFEFFFEFDFF00FF00FE0002000100
:1011000000020201010102020102010101000000CE
:101110000000FF0000FEFE00FFFEFEFFFFFFFFFDE0
:10112000FFFFFEFFFEFEFF00FEFFFFFFFFFFFFFFD2
:1011300000FEFF00FF00FFFF0000FF0002FF0000B5
:1011400000000000FF000000FEFF00FFFFFF00FFA7
:10115000FFFFFF00FF0000FF00FFFF000000FF0097
:10116000FF00FF00FFFF0001040203FC070A09ED76
:10117000BCEC09F40E1AEFEA11536D24EFCEACBBB0
:10118000FD1C1B08D5D7FCFD213E2B17EDDDDDE353
:10119000F00413101005F311070DF4C1F6E8010176
:1011A0001F502B11D4D7E5F3FAF80AFA0F08FB0504
:1011B000FDFC03FFFC00F100FF00130BFBF4FD0638
:1011C000051109010AE3E7DC0522F4FEF9161C0902
:1011D00002F204FBFBFCF4FDF7F6F6F905060A1033
:1011E000000C0EFEF8E9F8EDF8161104F6F7FD0311
:1011F000081001F8F1FD17E1D6F3062D270BEBE4FB
:10120000EBFD151B00E7F30414161008DDC8D7EF3B
:101210001D272415EBF301061E14F6DFD1E107109C
:10122000150AF6FBFF0905F9FC080C00F8F5F600B5
:1012300001FFFFF4FB08050A0D070501F4F7FAF8B2
:10124000FC00FCF904FCFB080B1208F9F1ECF805B2
:101250000A00FC0B050003FAF7F6FD04020800FC87
:10126000010A1005FDC9C6F0012B473110FAD1C1A2
:10127000BCEA2007F8F20A2F434529F3D4C2E4025E
:10128000F409E6DDE9EF0919282A11E9D9E000217E
:101290002713FEEDFAFA0016F0DBF6EFC7ED1B069A
:1012A0000D140A10160B0E191208F6E5E9D8DBEC3E
:1012B0000121181D110603DCD4C3D3050F17272500
:1012C000121915060C01E8DFE4F7182909EFDDD043
:1012D000E3EDF40507040D0E1111131A140C0AF8AE
:1012E000FAF7D1CEE4100E021B1704FE090A02F42D
:1012F000F6EFF2E2C5ED0C10193A351C09D6C8E23A
:1013000008102C24E2F6C6B51D39372806D4BFE3F1
:10131000C4DF1717281711FAFA0D2A4802D6C2C7D8
:1013200003F903312609E7D8E803242910FFE5DE95
:10133000FF04F5DDE0FA051C22FF0003E4CEE835EA
:101340003B17EBD0F11C453D0BCBC5E91BF5BAF4BF
:10135000110CFE071E0AF50C07E8E7E8101DF2EA7B
:101360000E11FC101703140FED0715F2E4EEDCC9A3
:10137000F518251C17FDD701FBFEFFD7E705EA0F7F
:101380004A291F0A04F1D9FA07042221FCDBB9C05B
:10139000E0133611FFE2E71118232508C7D3EC0448
:1013A000310BF01527220DF1F8EAEAE6D2EBFD1831
:1013B0003117F9E4E0FA000809070A0303E6E2FB43
:1013C0000D1A15171700FE11FEE3D6D4F0092622D8
:1013D000FCEAE3E8062D1BF9F6090AF9F5ED02111E
:1013E000FEECEA07111505D4DBFA151EF7FE2925D8
:1013F0000DEDE5EEE0F6170CF807160AF9EBE5DF60
:10140000EA05280B060EFC07FD0F131718F1D4D1BF
:10141000E6081104FEF8F804F8F400082029230473
:10142000ECE0DEE5F210100B0906010CF6CBE1FF53
:10143000182C220DE6D7E3EF1C22111205E7DAF291
:101440001520F4E2F8F9002327FBE4E9FBF1E804B6
:10145000131B2211FCF6DAD9EB0C1E0A13F8FA0E54
:101460000B10FAEDFAFB00FCD9EC060B1011271655
:10147000F6E8E3F4FDF1F1FD0811060C1F1A0CEC7F
:10148000DBEB0004FE060901F5FFFBF7EEE80A14AA
:10149000090C08F6FF0A110A0304F9EFE4F6FEF559
:1014A000FB0C1004080C05F3F0000B00F1F70A0D1B
:1014B000F3E9F6FB051F2414FCEEF7F1EFF4FC074B
:1014C000060D0AF3E4F2FD06191505FBFD0703F905
:1014D000F9F4FEFF0002F0F80406100AF8F1FC0B24
:1014E000120EFAEAF0F1F80406041113FCF7FC05F9
:1014F00008FAEEFC090101FBFBFEF9FD05121A04D6
:10150000EDE7E8F40012181003F9EEF2030405F910
:10151000FA0B06070AFCEFF50204FFFFFCFC0508C6
:1015200003000303FAF1FD0A02F0EFF805100909C0
:101530000C05EFE8FA0100FB08120B01F6F7010CAD
:1015400009FEF5F3F5F90303FCFF020404FF0408A8
:1015500009FFF2F3F2F7FF050204100D06FCF6FF97
:1015600002FDF9FAF9FC07060407FFFAFF00FCFB8D
:10157000F9F7FF02050703FDFCFFFE040F0E06F856
:10158000E9EBF905030401F6FF050509050604F575
:10159000F2FC0202010100FFFAFF02FE0301030058
:1015A000FBFCFAFDFD00070A0703FBF7F9FC040545
:1015B000FCF9F8FE07030200FE0205070700F7F634
:1015C000FA060BFAF2F70204FDFAFE02FE01070921
:1015D0000E07FDF7FAF9F2F803090D03F8FAFCFF1C
:1015E00001000303FFFBF9FC05070202FEFE0201F6
:1015F000FFFEF6FAFEFE0605020102FBF4FC010204
:101600000100000102FEFE040904FEFBFE00F9F6E3
:10161000FE030300FEFD030701FCF8FD02FF0307C4
:1016200003FAFB010304FEFAFE0200FF0100FEFDC7
:10163000FD00FFFE0001050502FEFBFAFDFFFE02B4
:101640000302FBF7FF050500FCFD050601FEFCF8A3
:10165000F8FD02040301FEFF010302FFFE0000FD8E
:10166000000101FEFDFFFCFBFE04070302FDFA0082
:101670000301FEFE0000FFFFFFFF0302FEFDFD0071
:10168000FFFEFFFEFE000302020201FDFAFEFFFF65
:10169000FEFF000000FEFF0001000000644C3C3D26
:1016A0004232363008FAF961DBA9DEA2CEA6BFAC21
:1016B000AED8B3DBD4B5DAD7CBEB00250BDDE21423
:1016C0000DE4FB0C0B0E151B070F32FCD8FE170E9A
:1016D00012030D4E2C253B252140314375394532EF
:1016E000153820F5FD04EBFDF2DBC8D9C08EA5A1AD
:1016F000ACB3B1C1CFD4BCBFC9C9C8E4E7CFECFA21
:10170000F20211EDFF10F20E26100D2D2C293533AB
:101710002F35323838353B323E38302F1C222515D4
:10172000141E1B1004FB02F9F7EDD0D7D0C8CFC2AE
:10173000C8C6B5B0ACB3A9A3B8B7BBC3C4D0E0DBCF
:10174000E7F1EF0C0309212B3A48504B4C4F4C4822
:101750005A63575F5650503837382B241F1B2013BD
:101760000305FBF4DDD6D3CADED0BABCB7AAA8AE57
:10177000ACB4B5B4C4C5C8D3D0D4DAE1EDEDFA0346
:10178000071314191E21292326343C383642494BAD
:1017900043454A3D3F3C3F4434332B241810110845
:1017A00004FFF8F3E8D9DAD6CDC6C2BFBCB8ABB0F7
:1017B000B7B4C0C8BDC8D1CED5DAE2ECEEECF3FDCB
:1017C00001071320201F282E323540474043484947
:1017D000463A3F42363130312619150D0A0AFAF8D9
:1017E00000EEE7EDEAE1D3D0D6D3C5C3C2B8B0B5B9
:1017F000BBB5B3BFC7C8D1D2D4E2E8E8F2FDFF0958
:1018000011161A202730373038413F3A3A413A3BD7
:1018100039393C35342E2726211D1616100809FDAE
:10182000F7F5F0ECEBE5E0E1D6D1D0CAC7C2C1BF15
:10183000C0C4BFBEC5C5C6CCCED6DDE2E5EDF9FE5F
:101840000205070D1011171F22252C2B2F353638B6
:101850003B403E3D40413D373A372E27231D150B77
:101860000706FEF6F1EDE5DFD9D6D3D2CCC7C9C362
:10187000BDBEC1C1C2C5C5C7CBD1DCE0E1E7EBF15C
:10188000F4FA03090A0C16151A1F2126282F3238DC
:1018900037363C3B3A37383330302C29231E1A1B5D
:1018A000140E0AFFFDFAF3F2ECE6DFDBDAD3CFCC5D
:1018B000C9C0BEBEBABCBBBDBFC1C5CDD2D3DDE3BE
:1018C000E6EEF7FB00090F161E1E23282A2D2E32E6
:1018D000353736383E39363738373233312E2922CC
:1018E0001F19130F0A05FEF8F4F1EBE5E4DDD7D478
:1018F000D0CDC9C7C6C5C3BFBFC0C1C3C8CACDD379
:10190000DBE1E2E8EEF3FC00050D12171D202529AE
:101910002A2E2F31363637373737343634302E2AA1
:101920002924201C17140D0903FFFAF5F3F0EBE549
:10193000E2DFDDD9D7D5D2D2CFCFD1CECED0D0D065
:10194000D1D4D7DBDCE2E8EAEFF4F8FB03070A10B6
:101950001317191C1E222425292A2C2C2D31313134
:1019600030302F2D2A28241F1A15110B0400FDF9E1
:10197000F5F0F1EEE9E5E1DFDBD7D4D4D1CFD0D07B
:10198000D0CFD1D2D4D5D9DBDEE3E9EDF1F6FA0040
:1019900006090D1116181C1D202322262728292A86
:1019A0002C29282827252323211E1B1915110D0A50
:1019B000090400FCF8F5F0EDE9E5E3E1DFDCDAD855
:1019C000D5D5D3D2D2D4D5D8DBDEE0E2E7EAEDF04C
:1019D000F3F8FBFE0306080B0F111516181B1B1D51
:1019E0001F2122222424242525232322211F1D1ADE
:1019F0001714100D0A060300FCF9F7F3F1EDEBE9FB
:101A0000E5E4E3E0DFDEDCDBDCDCDBDBDEDFE0E2E9
:101A1000E4E6E9EAEDF2F4F7FBFD0003070A0C0F38
:101A200011131515181A1B1C1D1E20212121201F02
:101A30001C1B1A181512100F0C09070402FFFDFBDE
:101A4000F8F6F5F3EFEEEBEAE8E6E5E3E3E1E1E2F1
:101A5000E2E2E3E5E6E7E8EAECEFF2F4F7F9FCFFAF
:101A6000010406080A0B0C0E101213141616181A8D
:101A70001A1B1B1B1B1A1A1918171412100E0B090C
:101A8000070502FFFDFBF9F6F3F2EFECEBE9E7E601
:101A9000E4E3E1E1E1E1E2E3E3E6E8EAECEFF1F3DC
:101AA000F5F7F9FCFF010406080A0C0E10111213D9
:101AB00014151517181818191918181716151412BF
:101AC000100E0C0B0806040200FDFBF9F7F5F3F10C
:101AD000EFEDECEAE9E8E7E7E7E7E7E7E8E9E9EA75
:101AE000EBEDEEF0F3F5F7FAFCFE00010305070855
:101AF000090B0C0D0E0F10101112121313131414E6
:101B00001414131211100E0D0B090705030201FF27
:101B1000FDFCFAF9F8F7F6F4F3F2F1F0EEEDECEC87
:101B2000EBEBEBEBEBECEDEEEFF0F1F3F5F7F9FAB5
:101B3000FCFD0002030507080A0B0C0D0E0F101028
:101B4000111212121212111110100E0D0C0A0907A7
:101B50000605040201FFFEFDFBFAF9F8F7F6F4F3BF
:101B6000F2F1F0F0F0EFEFEFEFF0F0F0F1F2F3F46C
:101B7000F6F7F8FAFBFCFDFE000102040406070874
:101B800008090A0A0B0B0C0C0D0D0D0D0D0D0D0C9B
:101B90000B0B0A09080706050403020100FFFEFDFE
:101BA000FCFBFAF9F8F7F6F5F4F4F3F3F2F2F2F2DB
:101BB000F2F2F2F3F4F4F5F6F7F9FAFBFCFDFEFFAE
:101BC00000010203040506070808090A0A0B0C0CA9
:101BD0000C0C0C0C0C0C0C0B0A0A0808070504036F
:101BE000020100FFFEFDFCFCFBFAF9F8F7F7F6F541
:101BF000F5F4F4F4F4F4F4F4F4F4F5F5F6F7F8F994
:101C0000FAFBFCFDFDFEFF000102030304040506D0
:101C10000607070808080809080909080808080746
:101C20000706060504040302020100FFFFFEFDFD96
:101C3000FCFBFAFAF9F9F8F7F7F6F6F6F6F6F6F627
:101C4000F7F7F7F8F9F9FAFAFBFCFDFDFEFFFF00E4
:101C5000000102020304040505060607070707083A
:101C6000080808080807070606060504030302011A
:101C70000100FFFEFEFDFCFCFBFAFAF9F9F8F8F8AA
:101C8000F7F7F7F7F7F7F7F8F8F9F9FAFAFBFCFCCA
:101C9000FDFDFEFFFF000001020203030304040533
:101CA00005050606060606060606060606060505D8
:101CB00004040303020101010000FFFFFEFDFDFC1F
:101CC000FCFBFBFAFAFAF9F9F9F9F9F8F8F9F9F97C
:101CD000F9F9F9FAFAFBFBFCFDFDFEFEFFFF00003F
:101CE00000010202030304040505050606060606B4
:101CF000060606060606060505040403020202019E
:101D00000000FFFFFEFEFDFDFCFCFBFBFAFAF9F90B
:101D1000F9F9F9F9F9F9F9F9F9F9FAFAFAFBFBFC29
:101D2000FCFDFDFEFFFF00000101020202030304AF
:101D30000404050505050505050505050505050456
:101D4000040403030202020101000000FFFFFEFE83
:101D5000FEFDFDFCFCFBFBFBFAFAFAFAFAFAFAFAD2
:101D6000F9FAFAFAFBFBFBFCFCFCFDFDFEFEFFFFB3
:101D70000000000101020203030304040505050538
:101D80000505050505050505040404030302020114
:101D9000010000FFFFFFFEFEFDFDFCFCFCFBFBFB6A
:101DA000FAFAFAFAFAF9F9F9F9FAFAFAFAFBFBFC93
:101DB000FCFDFDFDFEFFFF00000101020203030325
:101DC00004040405050505050505050505040404C9
:101DD00004030302020101010000FFFFFFFEFEFDFC
:101DE000FDFDFCFCFBFBFBFBFAFAFAFAFAFAFAFA45
:101DF000FAFAFBFBFBFBFCFCFDFDFDFEFEFFFF001A
:101E000000010102020203030304040404040405A4
:101E1000050505040404040403030302020101018F
:101E2000000000FFFFFFFEFEFDFDFDFCFCFCFBFBD8
:101E3000FBFBFBFBFBFAFBFBFBFBFBFBFCFCFCFCEF
:101E4000FDFDFEFEFEFFFF00000001010202020395
:101E50000303030404040404040404040404030347
:101E600003030202020101000000FFFFFFFFFEFE6C
:101E7000FEFDFDFDFCFCFCFCFCFCFCFCFBFBFBFCA0
:101E8000FCFCFCFCFCFDFDFDFDFEFEFEFFFFFF007B
:101E90000000010101010202020203030303030324
:101EA000030303030303030302020202010101000F
:101EB000000000FFFFFFFFFEFEFEFEFDFDFDFDFD3D
:101EC000FDFCFCFCFCFCFCFCFCFCFDFDFDFDFDFD4B
:101ED000FEFEFEFEFFFFFF00000000010101010207
:101EE00002020202020203030303030303020202CB
:101EF0000202020101010100000000FFFFFFFFFEDE
:101F0000FEFEFEFEFDFDFDFDFDFDFDFDFDFDFDFDFD
:101F1000FDFDFDFDFDFDFEFEFEFEFEFFFFFFFF00E1
:101F2000000000010101010102020202020202029C
:101F3000020202020202020201010101010000008C
:101F4000000000FFFFFFFFFFFFFEFEFEFEFEFEFEA5
:101F5000FDFDFDFDFDFDFDFDFDFDFEFEFEFEFEFEAB
:101F6000FEFEFFFFFFFFFF00000000000000010178
:101F70000101010101010101010101010101010151
:101F8000010101010100000000000000FFFFFFFF50
:101F9000FFFFFFFFFFFEFEFEFEFEFEFEFEFEFEFE5C
:101FA000FEFEFEFEFEFEFEFEFEFFFFFFFFFFFFFF4A
:101FB000FF0000000000000000010101010101011B
:101FC0000101010101010101010101000000000006
:101FD0000000000000FFFFFFFFFFFFFFFFFFFFFF0C
:101FE000FFFFFEFEFEFEFEFEFEFEFEFEFEFEFFFF0D
:101FF000FFFFFFFFFFFFFFFFFF00000000000000EA
:1020000000000000000000000000000000000000D0
:1020100000000000000000000000000000000000C0
:102020000000FF0000FEFCE80C190F0AE2071A2B63
:102030000CDC12FC11F9D4DFF0E0B700DEE904F1AA
:10204000FE03100B12FCF8FFFE2AF3F3340D2F17DA
:10205000302F2819FB1C0023DE05F1DADFABE0B3DB
:10206000F7D4E9F1D539EBFCEBF6FB0B34E1270CA7
:10207000064A23070C21EF3303C831EC001101FE9F
:102080001617BBFEE206F8CA14DAFCFE0906FEECDF
:10209000E8F8CA040CF6FB35010E1FE931DCD20664
:1020A000EDE8081704282103FEF5E50CEDEB11DD42
:1020B000150BE5111412022105E912DE0309FBF1EB
:1020C000EFFEE3F9DEF5F1F518FC0E23091915EF23
:1020D00011E8D8FFD4F404FC080B2DF00820EE1210
:1020E00012ECFE21E5F20DE30707F7F30CEBE80E27
:1020F000DF2519E811091903FCF2E40FF1E601FBF1
:10210000EF0B09031F15F80BFAE4F7E90118F4F9CE
:1021100018F1FC0AFEDFF706E418F7160AE927159E
:10212000030FF0E70EE2F5FDF7050AFD080CF71ABC
:102130000517EBFD0AEFF4E403E40CFEFD08E80EDE
:1021400001EC11FDEC04F8F6160AFC13FE03FC0486
:1021500000EF08F0060D1225020D0AF10E11E5FA46
:10216000F4E609FFF10100F90201F00E05E705EDC3
:10217000EEF0F8E9FC14F4200BF50D0CF007130059
:1021800018070F07FE13E90401F505F30BEA000633
:10219000F112FC03F1E7F8E4FEEA00030505F71489
:1021A000F510020E04FE20FD1CFB0209F301FC0EDB
:1021B000F2F2FEEB08FCFE04F7FF0108F80AECFF60
:1021C000FCF515F304FC07FE0A07F713EAFE06F018
:1021D0000307F20D05EF12FAF205FFFD0202FE0100
:1021E000FFFD01FDF40BFF0609F2FFF9F8FF0A02FB
:1021F00004F507FDF903FA10F20817FD09FAF704D0
:10220000F9FD0005FF0106F40E010111F203FFFFC5
:10221000FAF3FBF1F4F2FFF6FFF9F90FFD110406F2
:1022200005010AF20CF50510F308FA08050000FC98
:1022300007FD090403FFF700F406FBF600E908F8C0
:1022400003FFF714FB09000105F206FFF90AF70680
:1022500005FC0BF8FE020102FFFCFD02FF03FF0775
:10226000F90508F40FFEFB04F9FDFC02FAFD04F386
:1022700008FDFF02F403FB03F6FD06FC0301FE0468
:1022800009030802FB0303FEFFFD00000607040428
:10229000FA02FBF901FEFEFA02F8FD04F40302FA69
:1022A00002FFFCFF01FEFE030A050806FE0700030D
:1022B00000FBFFFB00F9FC00F9FE01FDFC03FE0042
:1022C00002FFF5FEFBFC05F7010402FF0403FF0B10
:1022D000060404FF000103010100F905FFFC04FAF4
:1022E00001FEFF030000FAF9FEFCFA02F9FAFFF61C
:1022F000040200000306020BFEFF02FE0200FEFACB
:10230000FE03FB0202FA0704FF04FEFA01FCFB02D3
:10231000FFFFFE00020201FEFE02FCFF03F601FECB
:10232000FA02FF02FD020000010202FD040101FFAA
:102330000301FE00FF03FDFEFEFD02FF01FF0101A0
:10234000F905FEFBFEF7FF0000FC01FFFA040002A6
:1023500002FE000401FC04FF010700010101FA0272
:1023600000F800FDFEFFFFFEFEFEFD0200FE020182
:10237000FFFF02000101FE0400FEFFFFFFFD02FD62
:102380000005FD0100FD01FE010001020001FFFB4F
:102390000001FE03FFFF0100010102FD0002FD003C
:1023A000FDFBFEFFFF0002FE01FEFD02FFFE01013C
:1023B000020204010203FF02FF00FEFEFDFC00FB1F
:1023C000FEFF01000103FE0201FF020001FEFF000B
:1023D000FE00FDFE00FFFF0200FF02FF0003FEFE05
:1023E000FFFEFEFEFEFD01FF000101000000FF02F6
:1023F000FF0000FF010102000001000100FEFFFDDF
:10240000FEFEFFFEFD00FCFF01FF000000030304D1
:10241000020102FE00FEFEFFFDFFFF00FFFFFFFEC8
:102420000000FFFFFFFE0001000100FE010000FFB1
:1024300000FFFF02FF010101020200FE0000000098
:10244000FF00FF01FE02FD0408F9030B04F2FBF597
:102450000203F105FCF90F13F8FFFBFA04FD07086E
:10246000FE08110008E8F8FEE704F6F60622081652
:1024700008FF15E3FDF3ED03F1020BEFF7FAFD0E94
:10248000FB06FDF10CFF0BFA020BF1080EF914EC40
:10249000091DD30EE4F316ECF8FCFC2FF6EA10F657
:1024A0001DF402F8EA0FF50DFEDC100B0001F1F847
:1024B000FC000601EE021800FCFBFE0CEB09EF012C
:1024C00007F5141005022B092DF0E311CE1B0EE3C6
:1024D000F5E70BDDFE15E014EF1210EB150A0DF514
:1024E000F1F504E504E7EA1F0429E2F50F0216FB03
:1024F000FE02D60D08F202CF03FCFB0106021125F5
:102500001302091CF70AFBFA03E8EEF5E7F3EEF60F
:10251000F700FCF13903150DF722EF1104E103F97F
:10252000F5FFF5FAFF05F30EF8D90707000BF909D7
:1025300019DB1D0EF419FF0EECFF10F107F003FB81
:10254000D30CF9FAFDF22103E80F0201111313E293
:10255000FA07F0F4EA08FBE420FBF227EE1A00E7A2
:1025600005EF13EA0B17E71DFFF10EDB0903DB1282
:1025700002001A0D1102FB10E6FDE3F207E802DE8D
:102580001D06F730F5FC1F000203EC1802EFFCF00B
:10259000F4EB06FAE6FBF8090BF71A12100BF80B2E
:1025A000F20A05F9F9F603F40FF1ED08E8FE06DB8F
:1025B00003050616EC06062014021410090903028E
:1025C000EDDB01DEEADDFD08DE1E04EB2012061461
:1025D000F13B0BE22FF5FCF2D802E6CCFAF7F6EF6E
:1025E000040FEE1907130D0035F9F81BEDFDEDE8AA
:1025F00012D9F90BF51EEFFD11F000FEFEFEFC10E6
:1026000002F20D1008F5010EEA16130202F410F69C
:10261000E5E9E8FFFBEAFD0A0A111CFF1020091496
:10262000EDED0CF3EAEFD8F409ED02FBF516220FFD
:10263000FB170F12FFED0CE0FCFCD502E5F20FF3E7
:102640001118110A091200FA0BF5F701E402E4F679
:102650001BE302F20623F819ED0C2EE706E1FC0F4E
:102660000114DEE90F02F8F7E90F000A06F80A0282
:102670002909D30708FE0CD619FDFD11E6E9E82962
:10268000ECF4FFF828FE0E0DEF180FFD07E1F61D24
:10269000DFE416E8FBFBFD04EE0FFF11F51F1ADC6B
:1026A0001CFE1011DC0DF4F0F2E1F3EF07FD040065
:1026B000011F0D05100D0B10F5F203F902E3E4F311
:1026C000E521F8F1030227F918FFFC1E0A07E9F4D7
:1026D0000BF5F9F5DE04FCF50BF40416F517F2031F
:1026E00037E80EF8FF01EC12DEF5FAF80BED040402
:1026F0000614EE0A04EE11080C0BFAFDFA0205F1BD
:10270000F3E60008EE0AEA1020F608EE0D0FF61FB9
:10271000F2F32501F3EAF907F1FEDCE806FD1DF00E
:10272000E72C1B2104E62FF8FE0FD2ECEA020CD1B5
:10273000E917FBFC090D0916110F16F1170CE2F24F
:10274000F7F3F8D6FB09E5120AF9041B0F05050497
:1027500012FE010CF1F3FDE6F4F8F701ED060C00B2
:102760001CF9FC15021100F8FEF20CF5F8F9E61759
:10277000FBF500FA1DF1FB1CE90C09F8FDF11C0347
:10278000E7F5060F01FDFEF90B000008DD04FDEF83
:102790000AF00B14F41E0CF317F703FFF4F7F3FB26
:1027A000F20203F8FBF80303FC0F0F031D060410ED
:1027B000EC0BEDE000F2F2F2F4FB060E010D14F763
:1027C000241501F0FE11E9FBF4F3F8FEF7F7EBFD39
:1027D0001A0DF8FC18030E06030CF10009D10208CB
:1027E000F20DD618F9F21FF30404050FF6FB0603E9
:1027F0000CEB0EF7F313F20EF8ED13E9F20EEF1CEB
:10280000EEF820F216F9010EF90CF701F8F413EBCB
:10281000F1F9F608F00B0EF60E0C0407FF0D0AEFA7
:10282000FAF605FCE703EBFB05FC03F1260AF41BB3
:10283000F40800F813F1F702F5F9F8FE00FC01FEC8
:10284000F5FD0112060216FD1AF6EE11DF0DFBDD95
:102850000CF0F8040409F908030C02FB0BFF000656
:1028600006F1FA040CE6F50BF00CEEFE11F1110A7C
:10287000F9FA012AE5F80EEC16F30F01E60F02FE55
:10288000E6E719FAE510FB020E0922F3031EFEEE3D
:10289000ED17F5E60AE7F6F0F124E5031CFA19FF57
:1028A0000611FF0412E4F405F101F7FFF700E40557
:1028B00008E71DFBF720FC0B08F921F70AFFE704E6
:1028C000E8FCF4F601F100FF0208FD1312F51AFA14
:1028D0001213DF17FBF1FAEDFAE5F718E6FF0A012C
:1028E00018F2100807FD011DF1FE0FED0700E005CD
:1028F000E0F701F108FF1103080A02190AFE06F9C0
:1029000009E9F10DD2FF0CEA04F2080CFC1508FBF2
:10291000FF220DE20213F9F7E8F8FBEB05FCFFF7E5
:102920001019F1F51C0AF604010CE9060DF1FBF192
:102930000CFCEDFEF60302FD0FEC071DF609FE0B85
:1029400017E80C04E704F1FBF1F109F2FC000C15A7
:10295000F91D11F517F00103E409F7EE00F3030484
:10296000F10B000103F6FE0F17FC0404FD02FEF953
:10297000F1F60CFDEFFAF80FF3080BFA08F309086B
:10298000F5050908FFFC11EC0009E800F20104EB71
:102990000A06F812FE0504F30D070503FFFBFA0D06
:1029A000F7F3FAF30A07E2F60C0214F30D08FB0C36
:1029B000020BF6FA13FFE6FC010CDC0203DF0B004E
:1029C00019E3F82C130101070DF20407CE03F603F7
:1029D000F3D81504F10B0D0A010C21F1001805EDD7
:1029E000E807EBF2F3F501EC1115FCF60C1305FE0C
:1029F000080A0006F303F7F601F2F10007F0F60803
:102A0000020F0EF709FD1412E30707F801F7FB00A8
:102A1000F30207F1FC0005F3F70C0E02FE13FF00B2
:102A20001606EAF4F803F7E907FBFC0A0AF6F101D7
:102A30001700010706FFF11BFAFBF4FD0EDD0D1078
:102A4000E503F20511D80C10040A040FF9020BF784
:102A5000F80100FFDCF0020C03E70AFE062CF8F98F
:102A600008FE1BFCE8F104FFFEFCF2FBF20E04F38F
:102A7000020C0BFFFB0D0DF704FEF8F4070AEAF752
:102A8000070BFEEDFD0EED0610F400F51300FD1C26
:102A9000F8FAFC0508FBF9FEF6EE0201EBFD16F470
:102AA00003FFFD0FFF131CEFFB15E907EDF308E330
:102AB00002FDEC0417FFFBFD1206FF060600FB1DDE
:102AC000EAF100FC0FF5EC12F4E411FEFAF0111338
:102AD000FAFF110CF9080AFEF6FC0401E104FEE815
:102AE000FBF4090602031106FE1A05FF00F4FCFDC3
:102AF00003FAEEF401FF02EAF31906FF13FBF31ADF
:102B0000FB11F9E71203F2F60EF101FAF9F6EA0FFA
:102B10000EF701050C1CF1FD06FD030EFDEAF002A7
:102B200005F2F3EF0BFC070CF70E021505EE0E0293
:102B3000FBFDF903F3F002EFF60B0504ED1917E8BE
:102B400012FC06FFEE1DF2010EEB00FC0107E4FC97
:102B5000FDFD02010AF2130E0103FF08FCFC14F450
:102B6000EBFAF015E1EA1CF5F9080CFC050D010B78
:102B7000FB090AE8FD07FFF5EE06FAE80B10F5027F
:102B800006FC06FB0807F10A1B00E20EFEF004F744
:102B900016E9F00CFBFEF4000DF3FF17F4060D131D
:102BA000FFF809FCFFE6EF14F2F6FDDE17FE08164B
:102BB000EE0F0C0610ECF519EA0EFEE7FEF410F726
:102BC000FA070502FAFDF9010DF40106F224FFF0FF
:102BD0001A0300FEF9F3F0EFFEFFF6EF0304061C04
:102BE000FD15FF111AE816EEEE04E8F7EBF6EFFD1F
:102BF00009FC150000210DFD090B07FBF303F5E7A8
:102C0000FCE7FEF8F41EEA01120B02100AFA11F6B4
:102C10000F01E2000BF9FDEFFCF6EE14F9E81608DF
:102C2000F509FA2909F7110C00E602F6F302EB02A6
:102C3000EAE227EBFB1BFD17F5F929FDFB10F80174
:102C4000F6FFF5F0FBF50AEFFA0BE4150EF515ECBF
:102C50001715EC1205FA09F9F6F8F8FEEEF8EF068A
:102C600001F609FB120B0C13F11205E918EDE00552
:102C7000FA0004E4FB12F403020C040116FCFD1438
:102C800005F6F9FDF5FDEEF018F2FD11F8FC0BFD6F
:102C9000FB0FFD0301FA000EFDFE02F303F609F639
:102CA000E60900FE0EEE010CFE0FEF10FC0D0EE229
:102CB0001BEDFC15D70602E609E30A12EC15020823
:102CC00004F01A07F10EFA00FDFF09E700FDF6F324
:102CD000DF17F2F91FFC1E02FD17040206F7F2F8D7
:102CE000FEF2EEFBFA01F103FE010908120D020AE1
:102CF00012F306F6F7FDF3EBFA03EB0004F50919FE
:102D000003FDF9120DFDFAFB11FEF200FEED0CF9C8
:102D1000EF04FB06F8FE011609F207F4F80F0902AA
:102D2000FA0508EF0FF3EA11E7FC04E207090105D1
:102D30000D15FA05FE070EF2FFF7F005F6F7F9EFAD
:102D40000BFA020AFA090B060A070A01F80DEBFE54
:102D5000F9ED08E6F40C06F9F3FE1C07050CFEF984
:102D60000915FFF5FB07F4F2F3FFEDF50CFAFBFE96
:102D70000B07FD180E02FEF617FAF314FADC080032
:102D8000E6EFF514F9F50B0BFF0A07090DFC0D0032
:102D9000E30E0DEC0AE6FC01EDF8F9FEF010FF0180
:102DA0001700071B010EFBF410E705F6E601F0F62D
:102DB00001FBFDFD07080815FD110C0114EFF9F9E1
:102DC000F002ECF7FAF70EF40116F4060BFC05021C
:102DD0000D07F8FD0504F9FAF5F606F7F801E90E16
:102DE0000FF50EF60014FB040B0207F6F908F6FCCB
:102DF000F7F3F4F30006F4FE100D02030FFB0B14BF
:102E000000F4FBF6F9FCE8FFFBED0301FD02021004
:102E10000308130907FD0805EFFD01F5EAEE05F5C6
:102E2000F906F00306F31E04FF1F0819F70A06E36C
:102E300002F3ECECE4F504F2FD0C030A20040A12A0
:102E4000051302FCFBF3E9F6F2F0F1FB06F8FF03D1
:102E50000F070919F7070BF30DF7FF03F101EEF95F
:102E600000F7FC0005F7FB010D08FA08080AFB094A
:102E700004ED0BF900F8EC07F7FBFAFDFAFA0E0780
:102E8000FC090CFE0D0CF902FFFEF8EA02F7FDFE4C
:102E9000F80AF3010907F60A11F710FDFC0702050D
:102EA000F5F3F300FBE61404F205FD05FA100DFC42
:102EB000FC0A0DF0F60903FAF7F902EEFA13F5F43D
:102EC0000BF805FE0318FB040D02F1020AF1F8FFEE
:102ED000FD01EE0401F105FA03F903140AF90A15DC
:102EE000FD03FB04FCEEFFF3EB03F603F6F30CFE2D
:102EF0000E070D0B0D0A01FFFB03FC00EBF1EFF7D2
:102F000000ED06F40718F6141301100CFFFAFAF49A
:102F1000FD04EEFDEFF105F207FBFF0B0505070AC7
:102F2000070F04FFFFF5FD06EFF3FDE907FBED04D6
:102F3000FA1405F807001A0BF90AFEFD0005F2EE77
:102F4000FBF4FBEFF60700FC1407030C0118F8FD77
:102F50000EF200F0FE07F1F8FAFDF0FE0DF7040F97
:102F600004FF020A0CFB010EF302FBF805E407FB69
:102F7000E9FCFB0CEF0B0F0506012003F40806F338
:102F8000FAF9F4F2F504F6F109FE03060315FD0B58
:102F9000070C00FE06E605FA00F3E80CEFF904FE64
:102FA00009FF0C0B03FB060EF40307F1FE04F10608
:102FB000FFF405EEFB06F908FE0B08F40DFD07FC17
:102FC0000309F111FDF9F9F50702EFF900F30BFE22
:102FD0000309FC040C0702FB0507F902F8FEF1FEE9
:102FE000FCF3FDF70CFF00000206FE0B0A020106CF
:102FF00000FAFFF4FAF7F603EAFE0B0401FF0EFEF7
:103000000502090BF30FFFF203ED01FDEC0903EFDD
:10301000F61303F8060C0802010407F70A04ECFE95
:10302000F803F7EF0DF0FDFC0808F018010904079C
:1030300014E90309F8F6FB00F0F701F9F7F50B05C1
:10304000FDFF110EFC19000CFE0005E100F1FDF082
:10305000EF0AF2FFFE1000FE1D0403060FFDF60945
:10306000F8FCF4FA02EEF7FE00EEF90EFC08FC1490
:103070000DF81CFD01FB0603E805F1FEF7EF05EE78
:10308000F80C050006FF0E0E0313F80407F60BE319
:10309000FA03E704E90A05EA0DFE1408FC0D010C29
:1030A0000606F9F10300EEF3FE0201EC050EF2084C
:1030B0000BF501080EFFFC000306F808EEF503FF10
:1030C00005E5FB07FE000705F405100209FF0805EA
:1030D000F10602EEEE09F500FAF80BEF0A0302071B
:1030E000010FFE090CFDFEF303F8ED06FFFBF5FAF8
:1030F00003FDFEFF0103091506F00913FC05EEF4BC
:10310000FFF00EFAF4F0070CEC0DFA000DFE0F02C2
:10311000F91B00F10DFEFFF3F202FEF0FDFAF0FCE8
:103120001207F50B0115FD041DF2FFFFFCFCFAEF81
:10313000FAFBEB07F7F209FF080E0A08FE0806077C
:1031400003FBF8FAFCFAF7F0F8FAF8FC09070304B5
:103150000A100C07F9F90406FBFDEEF9FDF703FB75
:10316000EDF915000509FA0F09000AF8010CFEEC4B
:10317000EE0EFCF9F3F905F800FBF60D140807FA5A
:103180000608020500F5F100FEF0FDF8F308F70A65
:1031900000F717060A060805F20209FAF8F2F8F82D
:1031A000F403FDF7030604FF080BFF020604FEFD0F
:1031B0000200F2FD01FDF6F608FBFC06FDF003112E
:1031C0000CFFF30E070104FF00FA02F8FDF9F20507
:1031D000F8F40C01F6040A090D0500FFF60B03FED6
:1031E000FCF102F8F504FCF50306FC0007050602F5
:1031F000FF0E03F1010402FFF8FCF101FCF20AF3F7
:10320000030EF50B070507F9020C04F4FFFBF902A6
:1032100001FBF2F6FD010103FAFB130D0502F512A5
:103220000800FEF9F9F109ECF0FD0105F3040805C9
:10323000030B08FD0C0900FFF607FAF5FBF5EFFAA2
:103240000CF7FDFB0807FC0E080401080BFEFEFF4F
:10325000FEEF000BE7EFF30700F50BFD04080F0A84
:10326000FB030B06F60706E8FFF7F8FAE808FAF49E
:10327000FE1006F6160802070707F9F70802F3FC26
:10328000F1F4F7F50FF6F00A0409030C0508110232
:103290000CF5F906EEF8FCF7F3EC0102F911050064
:1032A0000A0A0D0C010702FA02FDF4EBF3F500F730
:1032B000F705FD0C12FD0A0BFB11F9FF03F807FDE2
:1032C000F2F8FFF0FAF4FC07FE0B03F50F0E090508
:1032D000FB03030AF5FDF5F509F2F3FCFAF608061F
:1032E000FD0903080A030A01FFFD0100EAFC02F7D9
:1032F000F7F90100FE0402FE09060305FA1101FBBD
:1033000000F707E80902EC0AF70600F90D00F103DF
:1033100008FD00020806FA080CF3F90901F700F2AB
:10332000FCFDF60FEFF7070706000B02070206FF8A
:10333000FE0201F8E8F902F7F80101F70414F403BA
:10334000080811FAFB0207FA0202E7F804F5F50093
:10335000FB0407F9090A0A060203FF0DF7F5FFF857
:10336000FCFCFEF6F30503FEFF02040109FF140056
:10337000F912F20103EEFDFDF1FEFCF9FC0304027B
:103380000703080BFC0610FEF9F801F4FC05F0F544
:10339000FBFD05FC0202FC0B080EFF050FFFFDF90B
:1033A000FDF0F902FCF4F305FDF4020A04F90A0D3C
:1033B000080A0311EFF50BF6F4F800F1F503FCFA37
:1033C000FC020C03031105FB0A0605F9FB08E403E4
:1033D00008EEF8EB070FF5F8000A011609F10C06E4
:1033E00008FFFDF80000ED05FEEEFF00F60504FF06
:1033F000040501010D060100F5FF0FF6FAF9FEFEC6
:10340000F706E70000FF16F601070104090BFCF1BF
:103410000601F902FAFAF9F603FFF404F9010B0ABE
:1034200004FB0A0909FCFB02F1F800F6FBF3FD03BB
:10343000F4110DFA0203080CFD0504F40001F9F77C
:10344000FCF7FB08F7F902FC0C07050901FB05076F
:10345000F90403F2FA09FBF700FCFBFFFFFE00FE94
:10346000011205F913FAF20C11F8EC06FAFDFDF859
:1034700002FCFB0005F8FA0CFAFC16FFFB05050739
:1034800005F7FB06F4FDFAF4F704FBF0060E04FD65
:103490000801090EFB06FCF41004F2F1FAF5FF0C2A
:1034A000ECFC00060F03FDFD12010708F506FEF710
:1034B000FFF6FEF2F5FC0207F70A06050104020515
:1034C00005F8040201F801F4F40CF3FAFFF70B011C
:1034D00001080402F80E0FF502FEF60604F4F1FCF2
:1034E000F804FFF40804FC0D0BF508070202FF02C4
:1034F000FA01F4F201F5FF03EFFE0C09FE06FF03EB
:1035000011F7F90708F60304F200FBF30700F605CC
:10351000F8F8050DF9020F01FF0508FD03FD010391
:10352000F4FCF9F7FC04FBF10507FCFF0B0903FDB4
:10353000080BFEFFFFFDF6FE04F3F104F9FEFFFDAC
:1035400009FB070605FA040DF808FFFBFD09FDF26B
:10355000FAFD0DF1EA0702FB04FFFF040E0C00F96F
:103560000C07F702F8FEEEFE03EF00F9FB000B0577
:10357000FD08060A05FE0708FBF702F7EE02FAF857
:10358000F9FAFB0A0BF81008050F0100FDFD010117
:10359000EBEE05F701F2040BEE11060505010D0433
:1035A00004F504FDF507F0F203FFFDFAFEFD0BFB49
:1035B000FB08F9120601FC040CFA02F6FFF8F6FF0C
:1035C000F3FDFAFD03FDFA00110302080706FF0AE6
:1035D000F50103F205EEF7FFF7FDF705FE0205071B
:1035E0000E011001080BF3FFFCFEF7F7EFFF03EEEF
:1035F00002FFFA06050809060C05FD020AF4FDFDA6
:10360000F703EA05F9FC04F902F70D000007060BC1
:1036100000F70EF9F10FFFF8F3FE02FBFC01F9FFD2
:1036200007FF04F7011002FB0403FE05FC02FDF690
:1036300001F3FE00F7FE07FFFA06FE090AF50B0488
:10364000F713FAF701FAFEF8F8FBFDFA0C00FB0B92
:10365000FF010B0304FFF809FFF9FB02FBF6FEFB79
:10366000FCFDFE0605F70C0CFC0501050001FFF44E
:1036700000F9FB01F3F70502FBFF0004060803FF56
:103680000B04FDFDF90400F5F5FDFEF70AF5F70959
:10369000000CFE00060C00FE06F009FEF903F4FF24
:1036A00003FCF900F50209F702020602FD0EFE0214
:1036B000030205F207FCFBFCEF03FAF800FFFB0333
:1036C0000B0405020A0800FE0205F208F5EF01F1FD
:1036D00000F4020DFA07FC0A0DFC14FEFD010305BF
:1036E000F000F2FCF9FAFEFA02FC0F0105020601F5
:1036F0000308F30702EC04FEF4FCFB00F7040307E5
:1037000000FB0BFD05FF00FEF70B02FBFC02FAFCC1
:1037100004FFFEF7FD0300FB0405F5080FF90401A3
:10372000FF06F9FEFFFEF9FE03F8FDFCFEFD0003B7
:103730000207FF050D06FFFDFEFC04F9F4FCF30291
:10374000FFFA05F80909FA05070C02FFFC01FEFA69
:10375000FEF6FFFD01FBF8F70C05FD07F8010E066C
:10376000FCFCFF07FE01FAFEFBFE07F3FBFF06FC75
:10377000F50708FEFD03000601010AEF0110FBFD3D
:10378000EEFC020000F9FEFD0B07F602FF04050245
:1037900004F90607F8FA0DF5FBFFED11F7F90DF343
:1037A0000004030200040704030EF7F30BF5F7FE11
:1037B000F8F7F5000803F70808F7120B02FDF90FF8
:1037C00001F0F502EFFDFDF704F40C02FE0CFD0C18
:1037D00003060DF507F7F7FAF209F4FDFFF5060702
:1037E0000203FDFC14FFFE09F815FBF901F0FFF3DD
:1037F000FB05FA04FDFF020907FB08F30410F9FBBF
:1038000000FC0508EE01FAF90EF804F7FA0DF9F9D3
:10381000020C01FE00FE14F9FE06EF0B04FBF3F4AC
:10382000020004EF00010111FE06FC0905FFFBFC8C
:1038300004F505F8FDFDFC01F1F70B0AFEF90402A1
:103840000809F908F20706F705F10103F800FFF38C
:10385000FF040009FBFE040506FC0801FCFB02094D
:10386000F1FBFC0005F500FEF90906F5020B01016C
:10387000FE040CFA04FCF605FFFFF0FB05FBFEFB63
:1038800004FFFB0B0DF8000B0301FE00F6FE02F92E
:10389000FEF6FBFDF80604FE010608000903FA0225
:1038A000FF01F8F30703F301FF02FAF60AFBFE1229
:1038B00001FB05000406FBFC01F9000CF4F605F51C
:1038C00003FFF801FE050A020004FF09F9FE0AFDE4
:1038D000F801F9FEFBF703F6FDFF1001FC07010AF2
:1038E0000200FE03F70903ED02F8FDFCF804FB00FB
:1038F00006FC0FFBFF0BFA08FCFB08FEFFFEF805B9
:1039000001EFF5F6030602FEFA0FF90A05F612FBBF
:103910000908EE0005F2FBFCF3FAF90010FAFB17B8
:1039200005FD030AFE0104FC01F401FBF5FDFCFFAB
:10393000F9020900F70B08FB0703F6020C00F8FC7C
:10394000FF07FCF10BF6F30E00F9FD0602FC05057E
:10395000FB050706FDF50704F0FD08F6F702FFF684
:1039600002060AF6F90E0200040802F8FF0BF2F153
:1039700005F9FC03F30301F40F04FF0803F808083A
:1039800000FFF3FC03FDF802F20006FA0201040551
:10399000000204FE00FB020400FCFFFFF9FE00022F
:1039A000FCF3FE0C07FB07FDFE08FA07FA0008FC13
:1039B000FFF90306F00004F70AF2F508FD0302031D
:1039C000000208090800F405FFF303F0F9FCFF0406
:1039D000F30204FC0C030110FF0507FD01FCF8EDE8
:1039E0000103EA0204F707FAFD10FF050B000207C6
:1039F00004FEF8FAFCFFF8F3FB0006FE0000F705F2
:103A00000E06FDFB080FFDF604F8F9FEFC02F604B5
:103A100003FB03FA0500F90F01F80804FA0102FF9D
:103A200001F00500F60401FCF409FEFD06FD0EFDA3
:103A3000F31102F7FFF90200FF01F5F80AFA030497
:103A4000F30103070000FCFD0CF80705ED0806F87C
:103A5000FAFD00FDF8FF09FC00FE06050010F7FA6C
:103A60000903FEFC03FBF7FEF905FAFB03F6050468
:103A700006FFFD0C08FE0801F308F70002EAF6FE57
:103A80000600FEFDFC0907FE0AFB0308FB08F9FF20
:103A900002F00204F304FAFE05FBFEFE01FBFF0444
:103AA0000507FC01070405F9FFFDFB00FFF8FC0119
:103AB000F4FE020001FDFF0E01050BF306050407ED
:103AC000EB0007EB04FDF3F8F60906FF001102FC1A
:103AD0001009F8FFFA0005F302F3EF09FDFE02F406
:103AE0000D09010DFFFE0204F8FE05F400FFFB07BF
:103AF000FBFB05F6FD0AFE06F9FB06010DFBF401D2
:103B0000060801F5F9F70506F8FBF40207FE0407BD
:103B100001FB030CF9FD07FB05FAF904F1F9FFFDC0
:103B20000201FB0302040FFC0607F70701FB02FB7F
:103B3000F2FB03F9FEF9F10C0CF90803FC0D06FF8A
:103B4000FFFE04FEFB04F8F6FAFD05F9F70301F3A6
:103B50000A0FFA050A050002FD04FAF308FFF1F85E
:103B6000FD02FC0106F403FF0606FE0A05FDFF0543
:103B700001FCFBFFF9FAFCFDFDF80305FD03FD0662
:103B8000FFFC16F8F907FB07FDFCFFF6FD0105FF3A
:103B9000FB01FA0208FAFFFFFC0BFE0003F60A0A1B
:103BA00002F9FC00FBFEFD00FBFA0101FB01090824
:103BB000F9FF0903FB0401F607F8FF00F3FF00011A
:103BC000FD05F8F80B0B00FD02FE0904FDFEF7F7FA
:103BD00009FCEF0106F5FF04FA0700060304FE03E3
:103BE0000DF600FEFFF8F800F307FEF90CF7FB05F1
:103BF00009010008FB0901FC09FFF405FDF3FEF3D0
:103C0000FB02F90701FF08FD0D010609FE03F70499
:103C1000FAFBFAF7FEF9FF00F90109FFFF060406B7
:103C200004040BF7FE0200FEF1FFFAF401FFFD01B0
:103C3000000603F60412FEFE03F90406F7FAFFF984
:103C400002FEF602FC0108FA02F80205FF0901FC77
:103C5000FD0C01FB07F1FF06F001FCF50602F90679
:103C600007F906070203FE07FEFFFBFC06F7FAFB57
:103C7000FCF70607F20403080B00FE0207FB01FF36
:103C8000F1FBFF02FDFCFBFB0AFEFF07FD00050246
:103C90000005FB0202F106FDFBFFFB05F704FFFD3B
:103CA000FFFF0AFCFE020105020303F6FE04FCFB13
:103CB00003FEFFF4FD0AF5FBFE09FD020CFA0BFF03
:103CC000020AF10105F6FCFC02FAF5FDFD0201FD18
:103CD0000307030A07FE0006FFFD07F7F800F303DA
:103CE000FAF20301000306FF08080101000AFDFBC8
:103CF00000F605FDF000FAFA02FEF70606FC0E0AD1
:103D0000FEFB040603FEF9FFF9FA00FBF7F90600D3
:103D1000F80A08FCFE040905FBFA04FB0002F700A0
:103D2000FB05FCF705FBFD02040301FD0407FE0390
:103D300006F800FEF60500FB01F7FC0BFD02FCF7A0
:103D40000404020003020104FD04FBF50CFAFFF673
:103D5000FA06F40305FEFB060202060604FFFBFF5B
:103D600007F8F806F8F207F7F902FD010307060560
:103D7000FD050DFFFCFFFDF8F7FFFBFAFDF9FD0661
:103D8000FF0206010905FD0002FFFF03F7F80CF230
:103D9000F708FFFEF500FE0601F70DFDFE0EFA0125
:103DA00007FC0200FF02FAFB04F8FDFEF503010028
:103DB0000103030500FC1200FC03F80602FCF6F602
:103DC000FD01FEF60504FA000000FF00FF00FE0101
:103DD000FDFC02FF01F50307F403FD0CF61345C3D8
:103DE000A8ED30575C3424F697DCDEC1E7FC24F9FB
:103DF0009FB0CA0E5F5C5C33380FF631ED01542B77
:103E000021079CA0BDB2FE1AE5E81200FC31525514
:103E10004B514249DA96283922EE8B9CA89BA6BCCE
:103E200008392B32DFC13D52434A4045FAA8E5012B
:103E3000C38F9CDAB18FB09BE45654541A094C4B93
:103E400044403E3C3C2F07B9859698C5C991A2A233
:103E5000B1DF1652504B503916F9053D453A2BD675
:103E600094929F999FADB7D8C3A7CE034162554F97
:103E70004D0C03322A15F4EDF8DBA5A3ACA8DC0247
:103E8000F1D6D6E51B3F3B5B60535531E4D0D9F901
:103E900026FFD1BBA9B2B3C0FD25332402F0EF2B1E
:103EA0005D56624F2605C3DE17F0E5DABFC0B5BA2E
:103EB000CBF82E3E3C26FF052337543D3138190EF2
:103EC000FAC9C7E8FD0CE1C4C7BAE10F263641457F
:103ED000371BFF0832473A270DEBDEE1F807EBE826
:103EE000F2D7C6CCEE30313B431D1611253D3124AF
:103EF000211103EDE2E0D7F7FEFBF8D8E5EBE8147B
:103F0000292A353337330E0B21292910FDDECDCF79
:103F1000DAF2F1E9F9F5E2ECF12143383E2B0B0F2F
:103F200021272B1700FAEED4C2C2D2E4F9F8F2F935
:103F3000F9141F192B29213022211EFFFB00F4EC5C
:103F4000E4D8C9B8CCEDF800FF0710121E212D31BE
:103F5000222813F1F1F7000CEEDDD2B7CAD7E0F456
:103F6000FC0C110C121A2128221E100405FFFFF868
:103F7000E3E1DFCBD7DDDDE4E1FE060418161B1715
:103F8000122323141002F7F1D4D9E2E5EEE5E0D4D0
:103F9000D0E9FE0B140A16190E1F1A14170A03F59E
:103FA000E0DEDFE5E7DADDDCDBF5FC040B030B0C20
:103FB0000B171811130D0A07F3EEE9DFD8D3E0DE73
:103FC000E3F7F6FCFDF90D1312170D0A0B03080BAE
:103FD00004FFF4EAE0D6E1E5E9EEE3EAF0F80C11DB
:103FE000181E140D04FE07060705F3F4F1EAEFE6C8
:103FF000E1DDE3F5F4F0FF060B110D1312121810BA
:1040000004F3ECF6FAF6F3E9E5E6E5F4F7F4F7F78E
:10401000000202121818201508FFF7FEFCFBF8E852
:10402000E5E3E6F3F1F1F6F90705010F0B0E1412C3
:10403000140E080E07FBEFE4ECECEEF1E3E9F1F609
:10404000070A090D0A0E0F0A1314131406F9F0EEED
:10405000F5F4F1EFE3E4EBF2020408101013100D95
:104060001211100C0503FBF6FFF8ECEAE7EBF1F395
:10407000FBFAFF090E161614120D0C07040C0700AC
:1040800002F4EAEBEEF7F7F5F8F4F5FB041112167B
:104090001B120F0B090F0902FEF7F4F0F3F9F4F10C
:1040A000F3F5FAFA010B080E17131414121109068E
:1040B00001FBF9F6F7F3E8EAF2F60203040802045A
:1040C0000C0E131517160D07040102FCF7F1E8EDAD
:1040D000F0F2FDFDFF05060B0B0C13111210080981
:1040E00008080C02F9F5EEF2F3F1EFF0F9FF070E14
:1040F0000B0E13101210090C0B0A09FDF8FAF9FA4D
:10410000F7F2EEECF4FB0007070C100E131212137B
:104110000E0A03F9F9FAFCFCF6F4F4F1F7FAFDFFE4
:10412000FF080B0C11101115100D060102FDFBF913
:10413000F0EEF2F6FDFAFAFDFE06080A0E0C0F0F7D
:104140000C0E0A070A03FDF8EFF1F1F2F9F5F7FD9D
:10415000FE04080B0D0A0B0C0B0D0A0A0A01FFFCEA
:10416000F6F8F5F4F7F1F0F6FB0305080D0C0D0A6F
:104170000A0C0708070203FFFAFDF8F3F3F2F6F85A
:10418000F9FDFC0105070D0D100F080805010303DB
:1041900000FDF6F5F6F5F7F7F9FBF9FCFE01090A63
:1041A0000E110B0908050602FFFCF8F8F8F7F6F502
:1041B000F6F7F70000FF0404080B080B0C0B0B06C6
:1041C00001FCF7F9FAF8F3EEF3F7F7FEFF0004024B
:1041D0000506050A0B0C0C060200FEFDF8F6F4EFCE
:1041E000F2F4F4F9FBFF03040708080B07070703C1
:1041F00004030201FBF6F4F1F3F5F5F5F4FAFF021E
:1042000007090B0B0809060204020101FBF7F7F688
:10421000F6F6F5F5F5F8FBFD0003090A090B0A07A8
:104220000702FEFDFAFAF9F6F6F6F6F6F8FBFCFDE3
:10423000FEFD0104040A0C0909040200FDFEFBF85E
:10424000F6F3F2F2F6FDFEFF00FE000000050607A1
:10425000070605030100FDFBF9F5F6F3F2F6F8FB9E
:10426000FDFE020302050404040304050401FDFE2F
:10427000FDFAFAF7F4F4F3F6F9FAFF010205050581
:10428000050506050200FDFEFEFCFDFAF7F6F3F754
:10429000F7F6FBFDFF000206070709080603FEFE0E
:1042A000FEFCFBF8F8F8F7F9F8F6F7F9FDFF010462
:1042B000060708080705030301FDFAF6F5F6F7F906
:1042C000F7F7F8F9FDFFFF030405060707060505E4
:1042D0000400FCF8F7F6F6F7F5F6F8FAFFFFFF0230
:1042E00002040505050504030201FEFDFDFBFAF9C4
:1042F000F8F8FAFCFEFF00010102020202020100CE
:104300000000000000020203040404050208EEF3AA
:104310002C00C63B20C521F80822EF3C45E6FA08F0
:104320009ECEBB90D0CAFC0E244319FFEDDAC3CB5E
:10433000E5E5FB4957302FEADDDCA3D9EED3EC29C4
:104340003A494B1D3815DE0210FF010411323723A4
:104350000C0EF0CEDCDD050AF52F383F371A2E1093
:10436000E6EEF5F3FDFEFF04FCEFE8E4D3C0B2C9CE
:10437000D1D9EBE9F9E8DEF2EE0002E0F20AFD192C
:104380002E170DFC000B1016090C1624353F391999
:104390000A111309F2E5EAEBF00709F4F2EBDEDCAF
:1043A000D0CFCAC5E9040C1506F8F8F7F9F2EDF21A
:1043B000EF01233E44331F05FB02FFEFF80C091900
:1043C000303323FEEBE9E1E7F60506FA080F0C08A7
:1043D000F4E9E6E8EEF6070AF8F4F4EFF5F2ECF4A7
:1043E00003040001FCF2DFDDF401102336321F1D4F
:1043F0001505F0E6EAEAF5040C0E0E03F9F3E7E31F
:10440000E4E3E6F0011422221C0CFBF4EEF5FFFBC2
:10441000FBFD051310080402FCFA060B0601090D4A
:104420000C08FEF9EFE9F50105FF0106F8EDEFF2E2
:10443000EFEFF809100F0A0701F5FEFDFB0202037A
:10444000FCFE06090A03FF0807070A0502F7F3F94D
:10445000F7F5F3F7F9000905FBF4F1F0F1F5FB02CC
:10446000040A120803FFF7020A0B0D05FF080C08E7
:104470000902FF00FE01050C0C0D0F120DFEF4EDFC
:10448000EAECF2F6000B04FCFAF4EEEAE8ECF1FCDC
:104490000B0A0C0803060100000204050B110B00B7
:1044A000FBF9F7F6F5F7FA0106090E090400F7F82B
:1044B000FCF8FC04070B0B03FAF8F8F6F7F9FBFC21
:1044C00001080A0F0C04020002FDF7FB01070806B1
:1044D00008060301FCFBFBFBFBF6FAFDFE020606E9
:1044E0000504FFFAF6F2F3F6F9FC000304020000FB
:1044F000FEFBF7F7FCFF04090C080504FEF9F9F9C7
:10450000FC0002070A0809030000FCFAF9FC020497
:10451000060402FFFBFBF9F9FAF8FBFE01060707A8
:1045200003FFFF00FDFD010404040603FFFDF9F78E
:10453000F7FAFDFBFE0102040100FFFCFCFDFF0099
:10454000FCFDFF01020102FFFE00FFFEFCFAFCFE83
:1045500000000103030303030100000100FFFF004B
:10456000040402030301FFFCFCFCFDFEFF0001014B
:10457000010200FDFFFEFF01020400FCFBFDFFFB4A
:10458000FE01FF00FFFF00FEFDFE00010002000033
:1045900002010000FEFDFFFF01FFFFFDFBFEFDFF2E
:1045A00002000102000204020202FFFFFFFEFF0000
:1045B0000001010201FF0000FF00000000FF0101F7
:1045C0000000FFFF010201000000FEFEFDFDFDFDF9
:1045D000FF0103030102010100FDFDFCFDFE0000DF
:1045E000FFFFFFFEFF00FDFDFDFE000102020301D3
:1045F0000001010100000101FFFEFDFDFEFDFF01C4
:1046000002020201020200FEFEFEFE0001010201A2
:10461000010100FEFCFCFCFCFDFFFF0000010301AA
:104620000100FF000000FFFFFEFEFF0000FFFFFF94
:10463000FF0002010100FF000000000000FF000079
:104640000001FF02FF00FE0101FE00FF02FF01006A
:10465000308400001004DF0A1D10A219C01D4A3763
:10466000863CC23F0808040804030208040302024F
:104670000201010804030302020202010101010117
:104680000101010004050702892F11241FBECFEF8D
:10469000D8E0DEBFCDBF25E0A4E7B1E001C01D92A8
:1046A000A538B207E1F711E0A0E0B1E0EAECF7E7E6
:1046B00002C005900D92A437B107D9F713E2C5E403
:1046C000D3E204C02197FE010E94B13AC434D1075D
:1046D000C9F70E9420330C94E33B0C940000EF9246
:1046E0000F93FC01628314824295407F2F70422B0E
:1046F0004383802F8295807FE82AE18200830F9197
:10470000EF900895CF92DF92EF92FF920F931F9355
:104710002FB7F894C0907703D0907803E090790396
:10472000F0907A032FBF6C0D7D1D8E1D9F1D4FB71E
:10473000F8940091770310917803209179033091D8
:104740007A034FBF0C151D052E053F0528F0601795
:1047500071078207930758F71F910F91FF90EF9011
:10476000DF90CF900895AF92BF92CF92DF92EF92F9
:10477000FF920F931F93CF93DF936C017B018B010B
:10478000040F151FEB015E01AE18BF08C017D1075B
:1047900059F06991D601ED91FC910190F081E02DE5
:1047A000C6010995892B79F7C501DF91CF911F913A
:1047B0000F91FF90EF90DF90CF90BF90AF90089552
:1047C000FC01538D448D252F30E0842F90E0821B17
:1047D000930B541710F0CF96089501970895FC019C
:1047E000918D828D981761F0A28DAE0FBF2FB11DF4
:1047F0005D968C91928D9F5F9F73928F90E008954C
:104800008FEF9FEF0895FC01918D828D981731F005
:10481000828DE80FF11D858D90E008958FEF9FEF59
:104820000895FC01918D228D892F90E0805C9F4F2F
:10483000821B91098F73992708958BE793E00E945B
:10484000112421E0892B09F420E0822F089580E0D3
:1048500090E0892B29F00E941D2481110C94000006
:104860000895FC01A48DA80FB92FB11DA35ABF4F05
:104870002C91848D90E001968F739927848FA6895F
:10488000B7892C93A089B1898C91837080648C93B3
:10489000938D848D981306C00288F389E02D808162
:1048A0008F7D80830895EF92FF920F931F93CF9394
:1048B000DF93EC0181E0888F9B8D8C8D98131AC05B
:1048C000E889F989808185FF15C09FB7F894EE8942
:1048D000FF896083E889F98980818370806480839F
:1048E0009FBF81E090E0DF91CF911F910F91FF90EA
:1048F000EF900895F62E0B8D10E00F5F1F4F0F7392
:104900001127E02E8C8D8E110CC00FB607FCFACF4C
:10491000E889F989808185FFF5CFCE010E94312495
:10492000F1CFEB8DEC0FFD2FF11DE35AFF4FF0821D
:104930009FB7F8940B8FEA89FB8980818062CFCF83
:10494000CF93DF93EC01888D8823B9F0AA89BB89C6
:10495000E889F9898C9185FD03C0808186FD0DC0B1
:104960000FB607FCF7CF8C9185FFF2CF808185FFD2
:10497000EDCFCE010E943124E9CFDF91CF91089590
:104980003FB7F89480919D0290919E02A0919F0262
:10499000B091A00226B5A89B05C02F3F19F0019643
:1049A000A11DB11D3FBFBA2FA92F982F8827BC0189
:1049B000CD01620F711D811D911D42E0660F771FB1
:1049C000881F991F4A95D1F70895FC0181858111AF
:1049D00011862381348145815681D901A41BB50BF1
:1049E0004217530718F0DA01A21BB30B97819923E2
:1049F00009F17081519780F0711110C061E06083FE
:104A00001282118260816623E9F024173507D1F004
:104A100036832583892F08957723A1F0A181B28160
:104A20006A0F7B2F711D72836183603D774068F34D
:104A30001082E8CFAB2B29F081E080833683258379
:104A40000895108208950F931F93DC01ED91FC915E
:104A5000119701E010E020E030E004C0000F111FCA
:104A6000221F331F6A95D2F7442339F00E2B1F2BD8
:104A70000D931C931F910F910895009510950E238F
:104A80001F23F6CFEF920F93CF93DF93A62FB0E0C3
:104A9000EC01EB81FC81EA0FFB1F4083AD01440F69
:104AA000551FEF81F885E40FF51F11821082ED810B
:104AB000FE81EA0FFB1F30813F7040E1249FE0013F
:104AC00011242C2F232B2083EC01ED81FE81EA0F92
:104AD000FB1F2081207F0F70022B00834E2DDF9162
:104AE000CF910F91EF900C9423252A9870E062FBF0
:104AF000882780F986608EBD0DB407FEFDCF8EB588
:104B000086E0660F771F8A95E1F76EBD0DB407FE4C
:104B1000FDCF8EB51EBC0DB407FEFDCF9EB52A9A03
:104B20008F708927982789270895CF92DF92FF9267
:104B30000F931F93CF93DF93DC01A657BF4FC1E9BB
:104B4000D1E040E0BC0162557F4F6C0123EBC20E07
:104B5000D11C51E012E103E085EEF82E2D913C913D
:104B60001197411116C0FB018081982F9D7F9130D4
:104B700009F434608250823008F43860F601808194
:104B8000982F9D7F913009F431608250823008F473
:104B90003260899199918217930741F1CE01029772
:104BA000FC0131832083952F941B80917603811122
:104BB000FCCF809175038111F8CF8091BC0084FDFA
:104BC000F4CF1093F3022093F4023093F502009394
:104BD000F202509376031092F1028091F1029062FA
:104BE000990F982B9093F102F092BC0052964130AD
:104BF00041F4DF91CF911F910F91FF90DF90CF9003
:104C0000089541E0ABCFCF93DF93FC014081518108
:104C1000862F90E02381222369F0C681C40FD52F0F
:104C2000D11D6881278130E0860F911D2817390733
:104C300008F4C901A581A40FB52FB11D4481489F77
:104C40009001499F300D11243C9326812F5F2683CC
:104C50003281231710F0231B268326814381240FE2
:104C6000231720F42583DF91CF910895231BFACFDA
:104C70000F931F93CF93DF93E42FF0E0F595E79523
:104C8000A62FB0E0342F3170C32F30E0D32FAA0FFE
:104C9000BB1FA80FB91FAE0FBF1F50963C91509776
:104CA000E22F8E01000F111F000F111F01C0EE0F28
:104CB0000A95EAF7E327CD5EDE4F5881E523E32727
:104CC0005096EC93DC0190968D919C91009759F051
:104CD000DC01ED91FC910280F381E02DDF91CF9119
:104CE0001F910F910994DF91CF911F910F9108951A
:104CF000342FDC0114964C91149746130CC018966F
:104D00008D919C91DC01ED91FC910680F781E02D65
:104D1000422F632F099408950F931F93CF93DF932E
:104D20002F70413051F0F0F0423009F1433039F149
:104D3000DF91CF911F910F91089570E0675F7F4FD2
:104D4000660F771FFC01E60FF71F0190F081E02D41
:104D500023838681280F25838281281748F3281B07
:104D60002583E6CFFC01E60FF11D22A3E1CFE62F5C
:104D7000F0E026952F5FEF55FD4F2083D9CF70E0EF
:104D8000DB01A757BE4F1C92660F771FFB01EE5A3F
:104D9000F94B05911491FB01EC5AF94B4591549153
:104DA00041505109EB01C758DE4F2F3081F4598330
:104DB0004883FB01E758FE4F80819181880F991F3E
:104DC000880F991F9183808381E08C93B1CF21114B
:104DD00003C019830883EDCFCA01801B910B019694
:104DE00034E0969587953A95E1F7289FF001299F41
:104DF000F00D1124E00FF11F9F012F5F3F4F5983EA
:104E00004883E258F94F84914217530790F2F90111
:104E1000E258F94FE49187FF08C0E7FD06C0FB01A7
:104E2000E758FE4F31832083C4CF2F5F3F4F8E2F33
:104E3000EBCFCF92DF92EF92FF92CF93DF93EC0113
:104E4000E62FF0E07796EE0FFF1FE80FF91F518372
:104E500040838EA59FA528A939A9820F931FCAA4B4
:104E6000DBA4ECA4FDA482332DE09207F0F40097BC
:104E7000F1F481E1C8168BE2D806E104F10471F087
:104E800081E19BE2A0E0B0E08AA79BA7ACA7BDA709
:104E90008BEA95E09093890080938800DF91CF9111
:104EA000FF90EF90DF90CF90089581E39DE060E068
:104EB00073E00E947E3AFB01EE0FFF1FE859F94FA5
:104EC00025913491FC01EE0FFF1FE859FF4FA5918A
:104ED000B4910E946F3A59E09695879577956795BA
:104EE0005A95D1F7E4E0660F771FEA95E1F79B0149
:104EF00050E040E02C153D054E055F0579F22AA7EC
:104F00003BA74CA75DA760E074E284EF90E00E94AD
:104F10004D3A3093890020938800C0CF08956111E5
:104F20000FC0DC011696ED91FC914483808591853C
:104F3000DC01ED91FC910190F081E02D642F09944A
:104F4000613071F4DC011696ED91FC91458380850A
:104F50009185DC01ED91FC910280F381E02DEECF93
:104F60000895EF920F93DC0118964C91B5E06B9F7A
:104F7000F0011124E255FF4FDC0114968D919C91B4
:104F8000EE24E39402E0242F68E08E0F9F1F0E941E
:104F90006F230F91EF9008950F931F93CF93DF939B
:104FA000FC016430D9F44E5D5F4F2FE0249FC001B7
:104FB000259F900D1124AC01452F55274695469508
:104FC00036E0440F551F3A95E1F760E086819781FE
:104FD000DF91CF911F910F910C9419276230A1F4AA
:104FE0002FEF3FE0241B350BA1E3BDE00E946F3A99
:104FF000AB01BC019CE076956795579547959A95CE
:10500000D1F7407E61E0E2CF61111DC04E5D5F4F80
:105010008FE0849F9001859F300D1124232F33272B
:1050200026952695838990E02817390708F4C90149
:10503000228D2817190611F0828F138EDF91CF91E0
:105040001F910F910895DC01A60FB11D1A968C9146
:105050008430A0F78F01080F111DD8015C969C9138
:10506000951761F3EA010680F781E02D2D2F482F77
:105070006481828193810E943826F801D48FDECF2B
:10508000DC0112968D919C91DC01ED91FC910280E6
:10509000F381E02D09940895DC0112968D919C9185
:1050A000DC01ED91FC910190F081E02D09947F925B
:1050B0008F929F92AF92BF92CF92DF92EF92FF9228
:1050C0000F931F93CF93DF93CDB7DEB7A0970FB6A3
:1050D000F894DEBF0FBECDBF8C01762E862F90E0F8
:1050E00080589F4F65E0880F991F6A95E1F72091DE
:1050F00076032111FCCF209175032111F8CF209167
:10510000BC0024FDF4CF9093F3028093F40282E07C
:105110008093F20281E0809376031092F1028091F5
:10512000F102806A8093F10285EE8093BC00809149
:1051300076038111FCCF8091BC0084FDF8CF80E222
:105140008093F20281E0809375038093F102809155
:10515000F102806A8093F10285EE8093BC00809119
:1051600075038111FCCF8091BC00982F9071E92EBE
:1051700084FDF5CF80E2E3EFF2E0DE0111960190CD
:105180000D928A95E1F7FE0131966F0158019E015B
:105190002F5E3F4FD80188248394408181814F3F07
:1051A00011F48F3F09F0812C90E0982F8827840F0D
:1051B000911D8D939D933296E217F30771F7912C11
:1051C000F601F088FFEFFF12812C2F2D2F7040E0A9
:1051D000692DC8010E9438262F2D207F30E094E0F1
:1051E000359527959A95E1F741E0692DC8010E9410
:1051F0003826F601F188FFEFFF12812C2F2D2F703A
:1052000042E0692DC8010E9438262F2D207F30E012
:1052100084E0359527958A95E1F743E0692DC8012B
:105220000E943826939482E0C80ED11C98E099120F
:10523000C7CF882001F1F501119211925F012FE093
:1052400040E06E2DC8010E94382620E041E06E2D1E
:10525000C8010E94382627E042E06E2DC8010E9456
:1052600038262FE043E06E2DC8010E943826E394D3
:10527000F8E0EF12E0CFF80172A2A0960FB6F89412
:10528000DEBF0FBECDBFDF91CF911F910F91FF9079
:10529000EF90DF90CF90BF90AF909F908F907F90D6
:1052A00008951F93CF93DF93EC01162F6E838885AB
:1052B0009985DC01ED91FC910480F581E02D099543
:1052C000111116C06F816F3F99F08AA9882381F070
:1052D0008A819B810E94572888859985DC01ED9100
:1052E000FC910084F185E02D6F8109958FEF8F830C
:1052F000DF91CF911F910895809171059091720572
:105300009093740580937305809163059091640573
:10531000FC0112AA60E00E945129E0916305F0911E
:10532000640582A9882311F08FEF8783809161053E
:10533000909162050C949525AF92BF92CF92DF9227
:10534000EF92FF920F931F93CF93DF93442309F4BF
:1053500061C0EC01EE81FF8182A9882309F465C058
:1053600066816F5F6F70CF010E945129888D998D82
:10537000880F991F9F8B8E8B198E188EEE80FF8061
:10538000570182E1A80EB11C6701D0E0C0E0D50151
:105390008D919D915D01D7011296ED91FC9113972E
:1053A0008E01000F111FE00FF11F16964C91208106
:1053B000318102C0369527954A95E2F760E020FFDB
:1053C00002C0F60162A10E9403268823D9F090E072
:1053D000FC01EC58F94BE491DE01AF51BD4FEC9369
:1053E0008C59994BFC018491FE01E752FD4F80835B
:1053F000F801E753FD4F80819181F801E754FD4F9B
:10540000918380832196FFEFCF1ADF0AC830D10540
:1054100009F0BDCFDF91CF911F910F91FF90EF90D9
:10542000DF90CF90BF90AF90089581E082ABA4CF82
:10543000EF920F931F93CF93DF93EC01162F4985C3
:105440008C819D8122E0E22E01E0242F6FEF8255B6
:105450009F4F0E946F230E80DF81C02D8AA981118A
:1054600019C01F3F89F0612F8A819B810E945728B4
:1054700088859985DC01ED91FC910084F185E02D12
:10548000612F09958FEF8F83DF91CF911F910F913E
:10549000EF9008951F83F8CFCF92DF92EF92FF92A3
:1054A0000F931F93CF93DF93EC01AE81BF811596CD
:1054B000FC901597EC81FD8114962C91C22ED12C75
:1054C000E657FF4F81E090E002C0880F991F2A95B0
:1054D000E2F7918380830C811D8104561F4FF801F0
:1054E000428150E070E060E0838194810E94DC3B67
:1054F000F80111821082EC81FD81AE81BF8112968C
:105500000D90BC91A02DC601880F991FA80FB91F3F
:105510002D913C91E456FF4F31832083EE81FF8132
:1055200022813381820F931FFC01208131810F2C56
:1055300002C0369527950A94E2F78C819D818D549F
:105540009F4F20FF18C022E0FC0120838C819D81A9
:10555000EE24E394088529854FEF6F2D84569F4FE5
:105560000E944225DF91CF911F910F91FF90EF9004
:10557000DF90CF90089521E0FC0120838C819D81F4
:10558000E12C09852885E8CF6F927F929F92AF9298
:10559000BF92CF92DF92EF92FF920F931F93CF9320
:1055A000DF93CDB7DEB7A0970FB6F894DEBF0FBE7E
:1055B000CDBF8C01862FF801A681B78114966C911E
:1055C00014978111B2C00480F581E02D413021F49F
:1055D000E255FF4F82E090C0DF01AA57BF4F0D9008
:1055E000BC91A02D1A968D919C91813D974008F415
:1055F00098C0E255FF4F128281818F708083D8015D
:105600001496ED91FC911597E255FF4F81E0808350
:105610001696ED91FC9142815381262F30E020585F
:105620003F4F95E0220F331F9A95E1F77A01FE0173
:1056300031965A01B0E1AB0EB11C6F013A01CF01B6
:10564000D3019C9011967C91B2E06B0E711CD60137
:105650009C9211967C93B2E0CB0ED11C6A147B0411
:1056600079F76F0170E1C70ED11CD70150967C917C
:105670005097708B51967C91718BB2E0EB0EF11CC0
:105680003296EC15FD0589F7709176037111FCCF08
:10569000709175037111F8CF7091BC0074FDF4CF57
:1056A0003093F3022093F40220E2FC01A5EFB2E074
:1056B00001900D922A95E1F722E22093F20221E077
:1056C000209376031092F1022091F102206A209338
:1056D000F10225EE2093BC00FA0162A3698341E048
:1056E00050E064EF73E00E942B3AD8011496ED91DC
:1056F000FC91E255FF4F81E08083A0960FB6F894AD
:10570000DEBF0FBECDBFDF91CF911F910F91FF90F4
:10571000EF90DF90CF90BF90AF909F907F906F9071
:105720000895C8010E94182AE0CF813031F7E48043
:10573000F580413021F4F701ED54FF4F4BCFC70105
:1057400088579F4FFC0180819181FC018285938560
:10575000813D974040F1F701ED54FF4F1282818166
:105760008F708083D8011496ED91FC911597EA57BC
:10577000FF4F0190F081E02D248116968D919C9130
:1057800022FF07C060E00E945129C8010E944C2AF4
:10579000B4CFDC011296ED91FC9180E1DF011D9206
:1057A0008A95E9F7F2CF15964C91159712960D91BF
:1057B0001C91E62FF0E0EE0FFF1FE00FF11FE080DD
:1057C000F1806701042E02C0D694C7940A94E2F7D0
:1057D00096012095309581E090E0A0E0B0E0042EA5
:1057E00004C0880F991FAA1FBB1F0A94D2F7C0FCE0
:1057F00013C08E299F2991838083F80180A191A1F4
:10580000009709F47ACF2170DC01ED91FC910190B1
:10581000F081E02D099571CF809590958E219F2183
:10582000EACF1F920F920FB60F9211242F933F933E
:105830004F935F936F937F938F939F93AF93BF9398
:10584000EF93FF938BE793E00E943124FF91EF9158
:10585000BF91AF919F918F917F916F915F914F9188
:105860003F912F910F900FBE0F901F9018951F9290
:105870000F920FB60F9211242F938F939F93EF9354
:10588000FF93E0918B03F0918C038081E091910371
:10589000F091920382FD1BC09081809194038F5FF1
:1058A0008F7320919503821741F0E0919403F0E00B
:1058B000E558FC4F958F80939403FF91EF919F9152
:1058C0008F912F910F900FBE0F901F901895808190
:1058D000F4CF1F920F920FB60F9211242F933F9384
:1058E0008F939F93AF93BF938091770390917803A9
:1058F000A0917903B0917A0330919C0223E0230FA9
:105900002D3758F50196A11DB11D20939C0280935F
:10591000770390937803A0937903B0937A038091EF
:105920009D0290919E02A0919F02B091A0020196CB
:10593000A11DB11D80939D0290939E02A0939F0292
:10594000B093A002BF91AF919F918F913F912F9102
:105950000F900FBE0F901F90189526E8230F029608
:10596000A11DB11DD2CF1F920F920FB60F9211241D
:105970008F939F93EF93FF938091B900887F883234
:10598000D9F1D0F4803171F168F4882379F088304E
:1059900049F1FF91EF919F918F910F900FBE0F9062
:1059A0001F901895883141F1803299F784E98093EE
:1059B000BC0010927603EDCF803409F441C030F47E
:1059C0008033A1F3883329F785E9F1CF803559F188
:1059D0008835F1F18834E9F684E98093BC001092AF
:1059E0007503D7CF8091F1028093BB0085EC809343
:1059F000BC0010929B02CDCF90919B028091F2024D
:105A00009817A0F6E0919B02F0E0ED50FD4F8081E9
:105A10008093BB0080919B028F5F80939B0285ECFB
:105A20008093BC00B6CFE0919B02F0E08091BB0078
:105A3000ED50FD4F808380919B028F5F80939B028E
:105A400090919B028091F202981748F385E8E8CF85
:105A5000E0919B02F0E08091BB00ED50FD4F808310
:105A6000BBCF1F920F920FB60F9211242F933F932B
:105A70004F935F938F939F93EF93FF9389B180959B
:105A8000E0E5F6E49491982320919902921709F4A5
:105A90003CC0282F30E0E4E8F6E45491E5E8F6E471
:105AA0004491F90102C0F595E7955A95E2F7EE0F9A
:105AB000FF1FEE0FFF1FE470FF2702C035952795EB
:105AC0004A95E2F7F3E0220F331FFA95E1F72870C9
:105AD00033272E2BE0919702E695E695E22BE09393
:105AE00097020E2E000CFF0BE05CF94BE491209125
:105AF000E9023091EA022E1B3109E7FD339530931C
:105B0000EA022093E90290939902E1E5F6E42491F8
:105B1000282390919A02921709F43BC090E0E6E89E
:105B2000F6E44491E7E8F6E43491FC0102C0F5950F
:105B3000E7954A95E2F7EE0FFF1FEE0FFF1FE470A7
:105B4000FF2702C0959587953A95E2F753E0880FB5
:105B5000991F5A95E1F7887099278E2BE09198024A
:105B6000E695E695E82BE09398020E2E000CFF0BCD
:105B7000E05CF94BE4918091EB029091EC028E1B7A
:105B80009109E7FD93959093EC028093EB022093AB
:105B90009A02FF91EF919F918F915F914F913F9169
:105BA0002F910F900FBE0F901F9018951F920F927C
:105BB0000FB60F9211248F939F93EF93FF9383B1AE
:105BC0008095982F9170EEE5F4E090838695817032
:105BD0008183FF91EF919F918F910F900FBE0F9056
:105BE0001F9018951F920F920FB60F9211248F934A
:105BF0009F93EF93FF93809179009091960291305B
:105C000059F09230B9F1FF91EF919F918F910F90E0
:105C10000FBE0F901F901895E0919502F0E080580C
:105C2000EB56FE4F8083E0919502F0E0EB56FE4F7D
:105C3000808187FD16C0E0919502E150FF0BEB5685
:105C4000FE4F808187FF0DC082E080939602E09135
:105C50009502F0E0EB56FE4F808180939501109203
:105C60009502809195028F5F809395028EEC8093D0
:105C70007A00C9CFE0919502F0E08058EB56FE4FD4
:105C80008083809195028F3F21F483E08093960278
:105C9000BACFE0919502F0E0EB56FE4F808187FD90
:105CA000E0CFE0919502E150FF0BEB56FE4F808173
:105CB00087FFD7CF9091950280910201981788F2C3
:105CC00084E0E4CF78941F920F920FB60F921124C4
:105CD0002F933F934F935F936F937F938F939F93F4
:105CE000AF93BF93CF93DF93EF93FF9390E080E068
:105CF00050E040E0FC01E757FE4F60819C01220F1D
:105D0000331F6623D1F0D901A754BD4F0D90BC912C
:105D1000A02DE901C753DD4F68817981A617B70728
:105D200061F4D901A758BE4F6D917C91D901A75557
:105D3000BD4F11967C936E931082D901A754BD4F2D
:105D40006D917C91119727553D4FF901208131814B
:105D50002617370788F1ED91FC911197F695E79595
:105D6000F695E795E258F94FE4910E2E000CFF0BE3
:105D7000EC01CF51DD4F2881BF0102C075956795B9
:105D80002A95E2F7460F571FEC01C752DD4F2881D5
:105D900002C0F595E7952A95E2F74E0F5F1FFC01CB
:105DA000EF55FD4F20816D917C911197260F372F74
:105DB000311D11963C932E9301968830910509F080
:105DC00099CF40385105B4F08FEF8093B400FF9124
:105DD000EF91DF91CF91BF91AF919F918F917F9183
:105DE0006F915F914F913F912F910F900FBE0F9048
:105DF0001F90189540387FEF57071CF41092B4009D
:105E0000E6CF40584093B400E2CF909176039111D1
:105E1000FCCF909175039111F8CF9091BC0094FD47
:105E2000F4CF6093F3021092F40292E09093F202A6
:105E300091E0909376031092F1029091F1028062CA
:105E4000880F892B8093F10285EE8093BC00089522
:105E5000CF92DF92EF92FF920F931F93CF93DF9336
:105E600000D0CDB7DEB77C011A8219828B01085FA2
:105E700013406801D694C794D694C79442E050E08A
:105E8000CE0101960E941B3AC601880F991F880F08
:105E9000991FF801E81BF90BF695E7958601000FAD
:105EA000111F0C0D1D1DE00FF12FF11DFD96EE0FC2
:105EB000FF1FEE0DFF1D898190E0982F88272A8112
:105EC000820F911D9183808326E02C9DC0012D9D22
:105ED000900D1124E80EF91EF701E258FF4FD7018B
:105EE000A458BF4F8AE7E80EF11C8D919C91D70111
:105EF0002D913C91821B930B918380830F900F9087
:105F0000DF91CF911F910F91FF90EF90DF90CF9095
:105F100008958F929F92AF92BF92CF92DF92EF92AD
:105F2000FF920F931F93CF93DF9310927E031092F3
:105F30007D0388EE93E0A0E0B0E080937F03909330
:105F40008003A0938103B093820389E191E0909351
:105F50007C0380937B0385EC90E09093880380938F
:105F6000870384EC90E090938A038093890380EC0C
:105F700090E090938C0380938B0381EC90E090935E
:105F80008E0380938D0382EC90E090939003809336
:105F90008F0386EC90E0909392038093910310928C
:105FA0009403109295031092960310929703109207
:105FB0001E0410921F0410922004109221041092CB
:105FC00022041092230410922404109225041092AB
:105FD000260410922704109228041092290410928B
:105FE0002A0410922B0410922C0410922D048FE39B
:105FF00091E090935E0580935D0589E591E0909333
:10600000600580935F05809155058111CCC083E3C5
:1060100091E090939C0480939B0410929F041092B3
:10602000A1041092A0041092A3041092A20481E093
:106030008093A40490E19093A5048093A604109209
:10604000A7041092A8041092A9041092AA04109216
:10605000AC041092AB041092AE041092AD04809385
:10606000AF049093B0048093B1041092B2041092E4
:10607000B3041092B404E5EBF4E088E0DF011D9274
:106080008A95E9F7EDEBF4E091E08FEF1082128250
:10609000118214821382168215829783808711865B
:1060A0003A96B5E0ED30FB0789F788E0DF011D92F5
:1060B0008A95E9F7E5E1F5E08CE0DF011D928A952C
:1060C000E9F7C5E2D5E010E1198218821C861B862B
:1060D0001E861D861F86198A188A80E190E00E941C
:1060E000B73A9C01205F3F4FFC011192E217F30782
:1060F000E1F79C838B8380E190E00E94B73A9C019A
:10610000205F3F4FFC011192E217F307E1F79E83F6
:106110008D8380E290E00E94B73A9C01205E3F4F61
:10612000FC0111921192E217F307D9F798878F8338
:1061300080E190E00E94B73A9C01205F3F4FFC0154
:106140001192E217F307E1F79A8789871A8380E0B3
:106150009A81891738F4E985FA85E80FF11D808363
:106160008F5FF6CF6296B5E0C934DB0709F0ACCF9C
:106170001092490510924A0510924B0510924C0559
:1061800010924D0510924E0510924F051092500539
:106190001092510510925205109253051092540519
:1061A00081E0809355058BE994E09093620580939C
:1061B000610580919304811132C08BE291E090934C
:1061C000610480936004109264041092650410923C
:1061D00066048FEF8093670488E0EAE6F4E0DF016D
:1061E000282F1D922A95E9F7E2E8F4E0DF011D92DD
:1061F0008A95E9F710928A0410928B0410928C040D
:1062000010928D0410928E0410928F0410929004BC
:10621000109291041092920481E080939304C0E65E
:10622000D4E0D0936405C093630584E08093650552
:1062300088E080936605EBE0F1E0A7E6B5E0982FF3
:1062400001900D929A95E1F793E090936F0595E197
:106250009093700520ED37E030937205209371051F
:10626000309374052093730510927605109275058E
:106270001092770510927805E9E7F5E0DF011D92AD
:106280008A95E9F78FE595E0909369048093680417
:1062900083E290E00E94B73AFC0180E1DF01282F01
:1062A0001D922A95E9F79F01205F3F4FD9011D926A
:1062B0008A95E9F78FEF82A3D1A3C0A3F09363047B
:1062C000E09362048DE595E090939E0480939D0495
:1062D000F8942A9A229A8CB580618CBD8CB5806422
:1062E0008CBD239A259A8DB581608DBD8CB58D7F2F
:1062F0008CBD8CB581608CBD8CB58F7D8CBD8CB513
:10630000877F8CBD8CB58B7F8CBD68EF73E08BE98C
:1063100094E00E94282F6AEF73E08BE994E00E94DA
:10632000282F6CEF73E08BE994E00E94282F6EEF2A
:1063300073E08BE994E00E94282F55EBE52E54E0A2
:10634000F52ECBE9D4E010E001E099249A9466E0C0
:10635000862ECC24CA947FE0D72E5701F701808186
:1063600081113AC0812F8B7F612F09F058C18BE9D1
:1063700094E00E94752541E050E0143011F450E0A3
:1063800040E0B0E0A0E0849E9001859E300D112495
:1063900025563B4FF901E658FF4F40815181BC0122
:1063A000CD01641B750B810991094BE0660F771FC6
:1063B000881F991F4A95D1F722583F4FD9012D9137
:1063C0003C9150E040E00E94923ADA01C9019C5FA2
:1063D000AF4FBF4FB7FF08C01AA21CA21BA21EA23C
:1063E0001DA218A61FA20EC01AA21CA21BA28115D4
:1063F000E0E19E07A105B1050CF418C1DEA2CDA213
:10640000D8A6CFA209A79AA61BA6FFEFEF1AFF0AEC
:10641000D5018C91F701E95AFF4F5F01813009F0F6
:106420000AC1612F8BE994E00E94752521E081303B
:10643000984008F420E0D5012C931F5F2A9618306D
:1064400009F08BCF1092EC041092C40410927C00DF
:1064500080917C00806480937C0080917C008062CD
:1064600080937C0090E080E0812C912C54018394F7
:1064700030E020E0BC016C57794BFB01E20FF31FC9
:1064800044915AB17501640104C0CC0CDD1CEE1CB2
:10649000FF1C4A95D2F7C094D094E094F094452F15
:1064A0004C214AB9E4914BB17501640104C0CC0C94
:1064B000DD1CEE1CFF1CEA95D2F74C294BB92130AC
:1064C000310509F0BAC002968430910589F620980A
:1064D00028982198299856985E98539A5B98C3B14A
:1064E000C0958C2F817080935E048CE090E00E94B8
:1064F000B73AFC0113821782168211861086138622
:1065000012868BE9E82E84E0F82EF182E082128276
:1065100012E01583D1E0D483F0932205E0932105A6
:10652000C695C170C0935F048CE090E00E94B73ABA
:10653000FC0113821782168211861086138612863A
:10654000F182E082D2831583D483909324058093D3
:10655000230580916B00816080936B0080916B00BC
:10656000826080936B00D89A8091680081608093EC
:10657000680080916D00846080936D0080916D0053
:10658000806180936D0080916D00806280936D00CA
:1065900080916D00806480936D0080916D008068B3
:1065A00080936D00DA9A809168008460809368001F
:1065B00088E08093A50480919F0488301CF087E0D8
:1065C00080939F0478948091B9008E7F8093B90066
:1065D0008091B9008D7F8093B90088E48093B800E2
:1065E00085E48093BC0060E080E00E94052F61E0BC
:1065F00080E00E94052F60E081E00E94052F61E0AD
:1066000081E0DF91CF911F910F91FF90EF90DF908C
:10661000CF90BF90AF909F908F900C94052F8BE9F7
:1066200094E00E9475251AA21CA21BA29EA38DA312
:1066300098A78FA3E7CE108200CF21E030E01DCFD6
:10664000CF93DF9300D01F92CDB7DEB7789484B597
:10665000826084BD84B5816084BD85B5826085BD5E
:1066600085B5816085BD80916E00816080936E00EC
:1066700010928100809181008260809381008091DE
:10668000810081608093810080918000816080938F
:1066900080008091B10084608093B1008091B0004F
:1066A00081608093B00080917A00846080937A004A
:1066B00080917A00826080937A0080917A00816074
:1066C00080937A0080917A00806880937A0010929B
:1066D000C10010925A0410925B0410925C04109254
:1066E0005D0410921A0410921B0410921C04109264
:1066F0001D0468EB7BE080E090E00E9482230E9412
:10670000C0244B015C0198EEC92E93E0D92EE12CF8
:10671000F12C0E94C024681979098A099B09683EF6
:10672000734081059105A8F321E0C21AD108E10860
:10673000F10838EE830E33E0931EA11CB11CC11486
:10674000D104E104F10429F7E0918B03F0918C036B
:1067500082E08083E0918703F09188031082E091CA
:106760008903F0918A0380E1808310929303E09182
:106770008F03F091900386E08083E0918D03F09188
:106780008E03808180618083E0918D03F0918E0380
:10679000808188608083E0918D03F0918E038081F9
:1067A00080688083E0918D03F0918E0380818F7DDE
:1067B00080832FB7F8948091770390917803A0910C
:1067C0007903B0917A032FBF80931A0490931B042E
:1067D000A0931C04B0931D0440E150E063E671E017
:1067E0008BE793E00E94B3236AE070E080E090E0E2
:1067F0000E94822381E080932E04E0916105F09154
:1068000062058387868B81A30091630510916405DF
:106810008091B6008F7B8093B6008091B6008F7D0B
:106820008093B6008091B00081608093B000809129
:10683000B00082608093B0008091B100877F809328
:10684000B1008091B0008F7E8093B0008091B00045
:1068500080628093B0008091B0008F7B8093B00005
:106860008091B0008F778093B0008091B1008160FB
:106870008093B1008091B1008D7F8093B1008091B1
:10688000B1008B7F8093B100F894809180008E7F5F
:1068900080938000809180008D7F80938000809124
:1068A0008100886080938100809181008F7E809339
:1068B00081008091810081608093810080918100BE
:1068C0008D7F80938100809181008B7F80938100F8
:1068D0008091030190910401909389008093880036
:1068E00080916F00826080936F007894F80182A598
:1068F00093A5A4A5B5A581319B42A105B10579F069
:1069000081E19BE2A0E0B0E0F80182A793A7A4A7F1
:10691000B5A78BEA95E09093890080938800580191
:10692000F2E1AF0EB11C780122E2E20EF11CA0E10F
:106930007A2EBFE08B2E80E8982E88E090E00E94AF
:10694000B73A6C01DC0113961C92139715961C92B2
:10695000159716961C92169712967C9280E190E0FD
:106960000E94B73AF60191838083D501CD92DD92E2
:106970005D0187829482EA16FB06F9F642E556E449
:1069800089ECC82E82E0D82E61EE72E0A9EDB2E06B
:10699000570190E080E023E8822E26E4922E33E730
:1069A000632E36E4732EE4E05E2EFFE04F2EFA01F4
:1069B00025913491F6013183208332966F019C0139
:1069C000220F331FF901E753FD4F20803180220C45
:1069D000331C220C331C318220824E5F5F4FFA0140
:1069E000E590F490F1E0EF1AF108F901E755FD4F59
:1069F000F182E082E080F180EE0CFF1CEE0CFF1CC7
:106A0000F182E082E080F18027543D4FF901F1826C
:106A1000E082F4012491FB012193BF01F301249151
:106A20002D93FC01EF55FD4F5082F50141925F011E
:106A300001968830910509F0BACFD80114961C92BE
:106A4000149718968D919C91DC01ED91FC91019029
:106A5000F081E02D60E00995F8011582808591852F
:106A6000DC01ED91FC910280F381E02D60E009955D
:106A700060E0C8010E945129E0916305F09164052E
:106A80000281138141E050E064EF73E0CE01019692
:106A90000E941B3A69816770C8010E9457288DE5E2
:106AA00095E00E944C2A4091650580916105909186
:106AB0006205F2E0EF2E01E0242F64E082559F4F43
:106AC0000E946F23662463948FB7F89440917703F4
:106AD000509178036091790370917A038FBF809110
:106AE000ED029091EE02A091EF02B091F002F42E2F
:106AF000F81A8F0D911DA11DB11D8093ED02909389
:106B0000EE02A093EF02B093F002009161051091A4
:106B100062051801BAE12B0E311C6801E12CF80165
:106B2000E754FF4FFB83EA832801FAE44F0E511C20
:106B3000D1018D911D01772473947E0CF6013A9654
:106B40005F018111AFC04601F2E28F0E911C8E2DC4
:106B50008B7F6E2D09F07DC0C8010E94752541E034
:106B600050E024E0E21202C050E040E0B0E0A0E0DB
:106B700066E0649F9001659F300D1124200F311F46
:106B8000F901E658FF4F40815181BC01CD01641BE2
:106B9000750B81099109EBE0660F771F881F991F1C
:106BA000EA95D1F722583F4FD9012D913C9150E001
:106BB00040E00E94923ADA01C9019C5FAF4FBF4F9B
:106BC000B7FF35C0F60116A215A260E0C4010E940D
:106BD000E524882309F466C0D80112968D919C9112
:106BE000DC01ED91FC910480F581E02DD6019A96AF
:106BF0002C919A9795964D915C912F3FA9F034E096
:106C0000569547953A95E1F730E02F5F3F4F429F09
:106C1000B001439F700D529F700D1124AB0164E0D1
:106C2000569547956A95E1F76E2D09953BC08115FC
:106C3000F0E19F07A105B10544F0EFEFFFE0D601B9
:106C40009696FC93EE939597C0CFF60196A385A3F5
:106C5000BCCFC8010E947525F60196A385A36F2DB0
:106C6000C4010E94E5248823E9F0D60195964D9150
:106C70005C91B5E0EB1211C1EA81FB81808180FF5C
:106C800026C194E0569547959A95E1F7D20118965A
:106C90008C911897841709F434C319966C9219973C
:106CA00018964C93E72C6501B8E07B1241CFC09059
:106CB0006105D09062058601065E1F4FE12CF80148
:106CC00081918F018130E1F46E2DC6010E947525FE
:106CD00041E08130984008F440E0F801E95AFF4F64
:106CE0008081481769F04083D60112968D919C915E
:106CF000DC01ED91FC910284F385E02D6E2D099568
:106D0000E394B8E0EB12DBCFC0906105D090620550
:106D1000E6E8CE0ED11CB12CA12C8F2C912CD601E3
:106D20000D911D916D01F501E25AFB4F8081E62C1A
:106D3000E81AF801848181FFD8C0268137812F3F6E
:106D4000320739F0280D391DD80117963C932E9340
:106D50001697F801268137812431310508F4CDC01A
:106D60008D7F8483F8018581823009F4A2C18085FA
:106D700091858F3F980739F0880D991DD801199694
:106D80009C938E931897F801848187FF18C08085A3
:106D90009185883C910598F0838181110CC0808198
:106DA0009181DC01ED91FC910280F381E02DD8010D
:106DB00012966C910995F80184818F778483D801AC
:106DC00014968C91149783FF0AC018962D913C91CC
:106DD0001997283C310518F0877F14968C93F80199
:106DE000828593858F3F980739F0880D991DD801CA
:106DF0001B969C938E931A97F8018481982F91701B
:106E0000E916F9F082FF1DC085FD1BC02285338580
:106E1000203D3740B0F08062D80114968C931497CF
:106E200013968C91139781110CC08D919C91DC016C
:106E3000ED91FC910680F781E02DD80112966C91BE
:106E40000995F8018581E81609F457C0E582848127
:106E5000982F9170E916D1F013861286846084838E
:106E6000838181110DC080819181DC01ED91FC91C4
:106E70000190F081E02D41E0D80112966C910995C6
:106E8000F8018481982F9170E91237C082FDB5C056
:106E9000877FD80114968C93B8C0B6E0EB1217C068
:106EA000EA81FB81808181FF12C084E0569547957D
:106EB0008A95E1F7D8019A968C919A97841709F4EC
:106EC00020C29B966C929B979A964C93EBCEF801BE
:106ED00082819381DC01ED91FC910480F581E02DAC
:106EE000A3CEAA24A394B12C1ACF9581E91609F454
:106EF00039CF8260848317821682AA94AB2889F7DF
:106F0000A0906105B09062058501D12CC12C6C2D3B
:106F1000F601EE0FFF1FE751FD4F20813181D801AF
:106F20001D969C911D971E968C911E97891730F087
:106F300016963C932E9315971E961C92F801868503
:106F4000891710F48F0D8687D80115964D915C91A5
:106F5000169717968D919C919A01281B390B37FF34
:106F600002C02D5F3F4F3595279535952795211503
:106F7000310539F1F8015087478337FDA0C0648699
:106F8000F8018185882369F08481820F84832385B9
:106F90009285222309F49AC089170CF492C0891BA8
:106FA0008483F50182819381DC01ED91FC9106805F
:106FB000F781E02DD8011C962C911C9714964C91CA
:106FC0000995055F1F4FCA94CD2809F074C0009140
:106FD0006105109162055801E8EBAE0EB11CD501B8
:106FE0008C918F0D8C93712CF5018081803108F488
:106FF00076C0805180837394F7CFF8012285338562
:10700000283C310548F1877F8483F801E4808E2D88
:107010008B7C84838381811170CF80819181DC019D
:10702000ED91FC910190F081E02D40E0D8011296A5
:107030006C9109958E2D887309F05FCFF8018081DE
:107040009181DC01ED91FC910280F381E02DD8016A
:1070500012966C91099551CF83FD0BC08F7E84836E
:10706000F801848184FDCFCFD8011186108688680D
:1070700011CF20853185283C310518F08F7E84831F
:10708000EFCF87FF02C08F778483F801848180610E
:10709000848383818111E4CF80819181DC01ED9132
:1070A000FC910480F581E02DD80112966C91099530
:1070B000D7CFE58222CFCC24C394D12C28CF1486FD
:1070C0005FCF87FF6ECF890F84836BCF89171CF04A
:1070D0009150948366CF87FF64CF148262CF77206C
:1070E00009F49EC06801FCE9CF0ED11CE12C472CAD
:1070F000512CD60112968C911297E81608F05BC0BD
:107100008E2C912C1396ED91FC911497E80DF91D9E
:107110008081882361F11796ED91FC911897C40145
:10712000880F991FE80FF91F80819181840D951DAB
:10713000918380836D917C9111970E2C02C076957E
:1071400067950A94E2F715962D913C91D901A80D07
:10715000B91D4C91242F207F30E054E035952795C0
:107160005A95E1F760FF05C08217930750F4E39446
:10717000C0CF4F7050E084179507C8F3841B950B60
:1071800002C0821B930B918380832F3041F0609566
:107190007095462F41706E2DC6010E942325D601A1
:1071A0001396ED91FC91E80DF91D80818F3FF9F266
:1071B00081508083DCCFF801E255FF4F6281662366
:1071C00059F18481870D84837081B1812B2F207FB9
:1071D00030E044E0359527954A95E1F7A22FBF703E
:1071E0009381492F407F50E014E0559547951A95BB
:1071F000E1F7721302C0841738F47B130DC09F703F
:10720000891750F07A1342C0841B8483B0836F3F88
:1072100019F08FEF860F82833596AE16BF0671F692
:1072200080916105909162050E949525E09163052A
:10723000F091640582A9882399F080917505909159
:1072400076058F0D911D909376058093750520919D
:107250007305309174058217930710F00E947C2902
:107260008091780590916F058917A0F48F5F8093C6
:107270007805E0E0F0E0EF2B09F426CC0E941D2415
:10728000882309F41FCC0E9400001CCC891B848336
:107290002083BDCF8913EDCF909177056FEF690FF4
:1072A000683038F48DE595E00E94182A80917805C1
:1072B000DDCF83EF890F8830E8F490E0E3E8F6E46F
:1072C0002491FC01EF51FD4F2083E3E7F6E4249184
:1072D000FC01E752FD4F2083880F991FFC01E75303
:1072E000FD4F2081318187549D4FDC0111963C93E5
:1072F0002E93DCCF809170059813D8CF0E947C2903
:10730000D5CFE72C650114CCEF920F93FC0184815B
:107310009581A681B78115962C9162131DC0DC0161
:10732000AD54BF4F442381F082E08C9384819581DA
:10733000EE24E394008521854FEF84569F4F0E94F1
:1073400042250F91EF90089581E08C93848195817F
:10735000E12C01852085F0CF84569F4F0F91EF904F
:107360000C94232502970C948439EF920F93FC011F
:10737000A681B78115962C911597621711F120857A
:1073800012964D915C91139714968C9190E0880F12
:10739000991F840F951FDC014D915C91062E02C050
:1073A000569547950A94E2F740955095B42FB170E1
:1073B000EB2E84819581022F41E084569F4F0E94DD
:1073C00042250F91EF90089502970C94B5390297DA
:1073D0000C944C2A0C944C2A0F931F93CF93DF9359
:1073E0001F92CDB7DEB78C01DC011496ED91FC91B4
:1073F0001597E255FF4F128281818F70808314961A
:10740000ED91FC91E255FF4F81E08083698341E07B
:1074100050E064EF73E0CE0101960E942B3AC80160
:107420000E944C2A0F90DF91CF911F910F910895E8
:1074300002970C94EC39DC01CB01FC01F999FECFE9
:1074400006C0F2BDE1BDF89A319600B40D924150EC
:107450005040B8F70895DC01A40FB51F41505040CB
:1074600048F0CB01840F951F2E910E943C3A415069
:107470005040D0F70895262FF999FECF92BD81BDD7
:10748000F89A019700B4021639F01FBA20BD0FB662
:10749000F894FA9AF99A0FBE0895A1E21A2EAA1B3F
:1074A000BB1BFD010DC0AA1FBB1FEE1FFF1FA217B4
:1074B000B307E407F50720F0A21BB30BE40BF50BB1
:1074C000661F771F881F991F1A9469F7609570953A
:1074D000809590959B01AC01BD01CF010895A29FBD
:1074E000B001B39FC001A39F700D811D1124911D98
:1074F000B29F700D811D1124911D0895AA1BBB1B05
:1075000051E107C0AA1FBB1FA617B70710F0A61BA3
:10751000B70B881F991F5A95A9F780959095BC01C4
:10752000CD010895052E97FB1EF400940E94A93A00
:1075300057FD07D00E944D3A07FC03D04EF40C943F
:10754000A93A50954095309521953F4F4F4F5F4F49
:10755000089590958095709561957F4F8F4F9F4FBF
:107560000895EE0FFF1F0590F491E02D09940F93FD
:107570001F93CF93DF938230910510F482E090E067
:10758000E0918305F091840530E020E0B0E0A0E0D8
:10759000309799F42115310509F44AC0281B390B9D
:1075A00024303105D8F58A819B816115710589F1F7
:1075B000FB0193838283FE0111C0408151810281CE
:1075C000138148175907E0F04817590799F41097A5
:1075D00061F012960C93129713961C933296CF017A
:1075E000DF91CF911F910F91089500938305109320
:1075F0008405F4CF2115310551F04217530738F0B7
:10760000A901DB019A01BD01DF01F801C1CFEF0142
:10761000F9CF9093840580938305CDCFFE01E20FCF
:10762000F31F819391932250310939832883D7CF57
:107630002091810530918205232B41F4209107018F
:107640003091080130938205209381052091050136
:10765000309106012115310541F42DB73EB7409117
:10766000090150910A01241B350BE0918105F0912D
:107670008205E217F307A0F42E1B3F0B28173907EA
:1076800078F0AC014E5F5F4F2417350748F04E0F7E
:107690005F1F5093820540938105819391939FCF03
:1076A000F0E0E0E09CCFCF93DF930097E9F0FC019E
:1076B000329713821282A0918305B0918405ED0167
:1076C00030E020E01097A1F420813181820F931FD8
:1076D00020918105309182052817390709F061C092
:1076E000F0938205E0938105DF91CF910895EA013F
:1076F000CE17DF07E8F54A815B819E0141155105F0
:10770000B1F7E901FB83EA8349915991C40FD51F71
:10771000EC17FD0761F4808191810296840F951F1B
:10772000E90199838883828193819B838A83F0E036
:10773000E0E012968D919C9113970097B9F52D91E9
:107740003C911197CD010296820F931F20918105E4
:10775000309182052817390739F6309751F5109284
:10776000840510928305B0938205A0938105BCCF58
:10777000D383C28340815181840F951FC817D907D5
:1077800061F44E5F5F4F88819981480F591F518383
:1077900040838A819B81938382832115310509F07F
:1077A000B0CFF0938405E09383059ECFFD01DC010B
:1077B000C0CF13821282D7CFDC0101C06D9341503C
:0A77C0005040E0F70895F894FFCF61
:1077CA00FF0104700400008505800004020401041E
:1077DA000003040FF0000000005324B323E023A0A9
:1077EA00241124EF2303240000000078268C2600AD
:1077FA000000004C284B284B28402800000000C4F9
:10780A002AB127CC278F278E279C29EA39EA39B54E
:10781A00398439EC39FEFF0000E739E739E439B237
:10782A0039183A564D4450565F317C315F564D44B3
:04783A0050560A009A
:00000001FF
